:040000000CEF00F011
:0C000800D8CFFFF5FACFFEF54FEF12F055
:1000180000EE10F012EE7DF0F9EC02F005EE71F052
:1000280015EEE2F0F9EC02F000EEC6F011EE00F089
:10003800640EF66E000EF76E000EF86E5EEC39F088
:1000480005EE64F015EE71F09E0EF66E000EF76E7A
:10005800000EF86E5EEC39F0B1EF12F02207DB0605
:100068004907FB06A2098B096F09B409250A040A86
:10007800CC0952095E0A4F0A4A0A540A450A590A23
:10008800630AD50A6F0A880A140BAA0AC00AF90A71
:10009800ED0A920A7F0A53746172746564210D0A2D
:0400A8000000000054
:1000AC00FFFFD96AD950130DDE0EF324E96E010E51
:1000BC00F420EA6EEE68ED6A010ED92AD964F2D703
:1000CC001200FFFFEED71001FFFFD20EE16E010E02
:1000DC00E26E0101166B00EE0CF0E150E926E250E5
:1000EC00EA22EE50FF0AED10D8A443D000EE0CF03B
:1000FC00E150E926E250EA2210C1EEFF11C1EDFFFA
:10010C00E1CF17F1E2CF18F1010113511211D8B45C
:10011C000DD017C146F118C147F112C148F113C1F6
:10012C0049F10A0E4A6F4B6B56EC38F017C1E1FFE0
:10013C0018C1E2FF00EE0AF0E150E926E250EA2293
:10014C0014C1EEFF15C1EDFF00EE0EF0E150E926F3
:10015C00E250EA22EE6AED6A00EE10F0E150E92678
:10016C00E250EA22EE6AED6A16C1E1F50101165180
:10017C000AD0130EE126000EE222010E0101162B0D
:10018C001665A9D7FF0E1200FFFF9FD7FFFFD96E90
:10019C00130DDE0EF324E96E010EF420EA6EEE6808
:1001AC00000EED6A1200FFFFF2D7FFFF0101126F84
:1001BC00E1C5E8FF130DD20EF324E16E010EF4201D
:1001CC00E26EE1CF13F1E2CF14F100EE0EF0E1504C
:1001DC00E926E250EA22EE50ED10D8A415D000EE3C
:1001EC0012F01351E9261451EA2273C5EFFF1C0ECD
:1001FC00AA6FAB6B00EE12F01351E9261451EA22F0
:10020C00EF509BEC2BF001011251F6EC28F013C1CE
:10021C00E1FF14C1E2FF00EE0EF0E150E926E250DE
:10022C00EA22EE2A000EED2200EE0EF0E150E92655
:10023C00E250EA22EECFF3FFEDCFF4FF030EF45CB5
:10024C00D60ED8B4F35CD8B003D8010CFFFFAED7F0
:10025C00FFFFE1C5E8FF130DD20EF3240101156F6A
:10026C00010EF420166F00EE0CF01551E926165114
:10027C00EA22EECFC5F1EDCFC6F135EC35F000C07A
:10028C0017F101C018F1010100EE0AF01551E92631
:10029C001651EA22EECFC5F1EDCFC6F135EC35F0B3
:1002AC0000C019F101C01AF1010100EE0EF0155158
:1002BC00E9261651EA22EECF00F0EDCF01F0080E40
:1002CC0000241B6F000E01201C6F1D6B1E6B140E87
:1002DC00AA6FAB6B00EE12F01551E9261651EA220B
:1002EC00EF509BEC2BF015C1AAF116C1ABF1110E1E
:1002FC000101AC6F1BC1ADF11CC1AEF17CEC2FF058
:10030C001BC1C5F11CC1C6F135EC35F000C01BF1A9
:10031C0001C01CF10101170ECB6F010ECC6F080E42
:10032C00CD6FCE6B0EEC29F004EC2BF015C1E1FF78
:10033C0016C1E2FF00EE12F0E150E926E250EA228B
:10034C00FF0EEF6E00EE0EF0E150E926E250EA22CD
:10035C00000EEE6AED6A1200FFFF7BD7FFFFD96E2D
:10036C00D9CFE1F5E1C5E8FF130DE20EF324E96EF8
:10037C00010EF420EA6EEF501200FFFFF0D71801C7
:10038C00FFFF5DEC29F018C1E9FF19C1EAFFEF6E20
:10039C00E1C5E8FF130DE20EF324E96E010EF42023
:1003AC00EA6EEE06000EED5AE1C5E8FF130DE20E03
:1003BC00F324E96E010EF420EA6EEE50ED10D8A491
:1003CC0004D0C7EC29F0000E01D0010E1200FFFF83
:1003DC00D8D7FFFFE1C5E8FF130DE20EF324E96E59
:1003EC00010EF420EA6EEE50ED10D8A4C7EC29F003
:0403FC00E1C5E8FF70
:10040000130DE20EF324E96E010EF420EA6E000EE5
:10041000EE6AED6A1200FFFFE3D70601FFFF01015C
:100420000B0E406F010E416F080E426F436B71EC73
:1004300029F00BC1C5F10CC1C6F135EC35F000C097
:100440000BF101C00CF10DC1C5F10EC1C6F135ECC7
:1004500035F000C00DF101C00EF10FC1C5F110C1A2
:10046000C6F135EC35F000C00FF101C010F111C13B
:10047000C5F112C1C6F135EC35F000C011F101C073
:1004800012F101010B0E136F010E146F06C115F16D
:1004900007C116F119D801010A6F0A29D8A403D09F
:1004A000C7EC29F00DD001010A51130DE20EF3241F
:1004B000E96E010EF420EA6E0FC1EEFF10C1EDFFF0
:1004C000010CFFFFACD71301FFFF01011769D20E2A
:1004D000D96E010EDA6EF36A010110EE02F01351CB
:1004E000E1261451E22200EE0CF0D950E926DA5050
:1004F000EA22EE52E652E550ED18E7CFE8FFD8B415
:10050000EF18D8A43CD010EE06F01551E126165194
:10051000E22200EE06F0D950E926DA50EA22EE5047
:10052000E61808E1EE50E61805E1EE50E61802E1A3
:10053000EE50E618D8A420D013C1E9FF14C1EAFF99
:1005400010EE0AF0D950E126DA50E222E652EE52DD
:10055000ED50E518EFCFE8FFD8B4E718D8A40CD0D9
:1005600000EE10F0D950E926DA50EA22EE50ED10F4
:10057000D8A402D0F35039D0F3500101176F130EF5
:10058000D926000EDA22010EF32AF364A5D7010161
:100590001729D8B428D01751130DD20EF324E96EC1
:1005A000010EF420EA6EE9CF46F1EACF47F1E9CF38
:1005B00018F1EACF19F115C148F116C149F10A0E37
:1005C0004A6F4B6B56EC38F013C1E9FF14C1EAFFD8
:1005D000010110EE0AF01851E1261951E222EECF86
:1005E000E6FFEDCFE5FF010117511200FFFF6DD7C8
:1005F000EE6AEA50E262FCD7E950E162F9D71200F4
:100600005458540048544D00474946004347490058
:100610004A504700434C4100574156007465787476
:100620002F706C61696E0000000000000000000087
:10063000746578742F68746D6C0000000000000011
:1006400000000000696D6167652F67696600000042
:100650000000000000000000746578742F68746D5D
:100660006C0000000000000000000000696D616780
:10067000652F6A7065670000000000000000000040
:100680006170706C69636174696F6E2F6A61766105
:100690002D766D00617564696F2F782D77617665B1
:1006A0000000000000000000485454502F312E304C
:1006B00020323030204F4B0D0A436F6E74656E74DC
:1006C0002D747970653A20000D0A0D0A00474554D3
:1006D00000494E4445582E48544D00485454502F1C
:1006E000312E3020323030204F4B0D0A436F6E7464
:1006F000656E742D747970653A2000485454502FFB
:10070000312E3020353033200D0A0D0A53657276B4
:1007100069636520556E617661696C61626C650D17
:100720000A00485454502F312E3020343034204E9B
:100730006F7420666F756E640D0A0D0A4E6F74201B
:10074000666F756E642E0D0A000D0A0D0A004D438A
:100750004850537461636B2076322E313100444827
:1007600043502F476C65616E696E672E2E2E0042D6
:100770006F6172642053657475702E2E2E002020D8
:100780002020202020202020202020202020004366
:100790004F4D4D414E44532E43474900494E444529
:1007A000582E48544D0066747000706963000D0A3D
:1007B0000D0A0D4D434850537461636B2044656DC1
:1007C0006F204170706C69636174696F6E2076315F
:1007D0002E3020284D6963726F636869702054431E
:1007E000502F495020537461636B20322E30290DF5
:1007F0000A0D0A09313A204368616E676520426F2D
:100800006172642073657269616C206E756D6265DA
:10081000722E0D0A09323A204368616E67652064C2
:10082000656661756C7420495020616464726573FB
:10083000732E0D0A09333A204368616E67652064A0
:10084000656661756C742067617465776179206194
:100850006464726573732E0D0A09343A204368612B
:100860006E67652064656661756C74207375626E71
:100870006574206D61736B2E0D0A09353A20456E43
:1008800061626C652044484350202620495020472F
:100890006C65616E696E672E0D0A09363A204469EF
:1008A0007361626C652044484350202620495020E3
:1008B000476C65616E696E672E0D0A09373A2044F0
:1008C0006F776E6C6F6164204D50465320696D6187
:1008D00067652E0D0A09383A205361766520262077
:1008E000517569742E0D0A0D0A456E74657220618A
:1008F000206D656E752063686F6963652028312DF2
:1009000038293A20000D0A496E76616C69642069C5
:100910006E707574207265636569766564202D203C
:10092000496E7075742069676E6F7265642E0D0A6A
:10093000507265737320616E79206B657920746FD6
:1009400020636F6E74696E75652E2E2E0D0A00255C
:1009500075000D0A4E6F772072756E6E696E672096
:100960006170706C69636174696F6E2E2E2E000D5C
:100970000A44656661756C742047617465776179B6
:1009800020416464726573732028000D0A44656613
:1009900061756C74204950204164647265737320E2
:1009A00028000D0A53657269616C204E756D626591
:1009B000722028000D0A44656661756C74205375B9
:1009C000626E6574204D61736B2028000D0A5265BC
:1009D00061647920746F20646F776E6C6F6164203E
:1009E0004D50465320696D616765202D2055736514
:1009F00020586D6F64656D2070726F746F636F6CDB
:100A00002E0D0A000D0A444843502026204950204C
:100A1000476C65616E696E672064697361626C65BD
:100A2000642E0D0A000D0A444843502026204950E8
:100A300020476C65616E696E6720656E61626C65EA
:100A4000642E0D0A00504F52540051554954005025
:100A50004153530053544F520041424F520055539B
:100A60004552003232302052656164790D0A0032FD
:100A70003330204C6F6767656420696E0D0A003261
:100A80003030206F6B0D0A00323231204279650D13
:100A90000A00323236205472616E736665722043EA
:100AA0006F6D706C6574650D0A00353032204E6FC5
:100AB0007420696D706C656D656E7465640D0A00F7
:100AC000353330204C6F67696E20726571756972BD
:100AD00065640D0A003333312050617373776F7290
:100AE000642072657175697265640D0A0031323572
:100AF00020446F6E652E0D0A00313530205472612E
:100B00006E7366657272696E6720646174612E2E01
:0C0B10002E0D0A00353030200D0A0000C8
:100B1C00FFFFD96AD950220D1C0EF324E16E000E92
:100B2C00F420E26EE76A00EE21F0E150E926E25093
:100B3C00EA22FE0EEF1600EE21F0E150E926E2501B
:100B4C00EA22EF50FD0B0209EF6E00EE21F0E150AE
:100B5C00E926E250EA22EF50FB0B0409EF6E00EE9F
:100B6C0021F0E150E926E250EA22EF0EEF1600EEFA
:100B7C0021F0E150E926E250EA22F70EEF1600EEE2
:100B8C000FF0E150E926E250EA22FF0EEF6E00EE84
:100B9C001FF0E150E926E250EA22580EEE6E020EEA
:100BAC00ED6ED92A040ED964B5D70001106B116F04
:100BBC00146B156B166B176B1200FFFFAAD7010194
:100BCC00FFFFD96AD950220D1C0EF324E16E000EE2
:100BDC00F420E26EE750010ED8A443D0E76E00EE8D
:100BEC000BF0E150E926E250EA2201C1EEFF02C10E
:040BFC00EDFF00EE1B
:100C00000DF0E150E926E250EA22EE6AED6A00EECC
:100C100007F0E150E926E250EA22EE6AEE6AEE6A57
:100C2000ED6A00EE21F0E150E926E250EA22EF50B1
:100C3000FE0B0109EF6E00EE21F0E150E926E250D3
:100C4000EA22F70EEF1600EE0FF0E150E926E2502F
:100C5000EA22FF0EEF6E00EE21F0E150E926E250AD
:100C6000EA22EF50FD0B0209EF6ED95005D0D926CC
:100C7000040ED964ADD7FE0E1200FFFFA8D70701FE
:100C8000FFFFD96A01010B6B01010B51220D1C0EF4
:100C9000F324E16E000EF420E26EE750010ED8A4BA
:100CA00002D0D96E05D001010B27040E0B65ECD7DD
:100CB000D950D8A402D0FE0EB3D00001102B000EE4
:100CC000112300EE0BF0E150E926E250EA2210C0B9
:100CD000EEFF11C0EDFF130E115D890ED8B4105D4B
:100CE000D8A003D0106B040E116F00EE21F0E1507C
:100CF000E926E250EA22FE0EEF1600EE0DF0E1507A
:100D0000E926E250EA2209C1EEFF0AC1EDFF000127
:100D1000142B000E15231623172300EE14F0E150B8
:100D2000E926E250EA2214C0EEFF15C0EEFF16C01D
:100D3000EEFF17C0EEFF00EE18F0E150E926E2509A
:100D4000EA22EE6AEE6AEE6AED6A010EE124010122
:100D5000466F000EE220476FE1CF0CF1E2CF0DF1BC
:100D600007C148F108C149F10A0E4A6F4B6B56ECB6
:100D700038F00CC1E1FF0DC1E2FF010EE1240101D9
:100D8000726F000EE220736F00EE0BF0E150E92667
:100D9000E250EA22EECF74F1EDCF75F100EE0DF0E6
:100DA000E150E926E250EA22EECF76F1EDCF77F17D
:100DB00000EE14F0E150E926E250EA22EECF78F19D
:100DC000EECF79F1EECF7AF1EECF7BF100EE18F0B5
:100DD000E150E926E250EA22EECF7CF1EECF7DF140
:100DE000EECF7EF1EECF7FF1020E806F8169826BD4
:100DF000836B0FEC0BF00CC1E1FF0DC1E2FF030EA2
:100E0000E76E00EE14F0E150E926E250EA22EE2A05
:100E1000000EEE22EE22ED22ED52ED5201010B51B9
:100E20001200FFFF2ED7FFFFD96E220D1C0EF324F8
:100E3000E96E000EF420EA6EEF50040A000ED8B4FA
:100E4000010E1200FFFFF0D7FFFFD96E220D1C0E1E
:100E5000F324E16E000EF420E26ED9500101666FBA
:100E6000E1CF67F1E2CF68F1E750040AD8B407D0C8
:100E700067C169F168C16AF1DCEC0DF057D001017E
:100E80006651DFD967C1E1FF68C1E2FF010EE124CD
:100E90000101726F000EE220736F00EE0BF0E15063
:100EA000E926E250EA22EECF74F1EDCF75F100EEC3
:100EB0000DF0E150E926E250EA22EECF76F1EDCFD7
:100EC00077F100EE14F0E150E926E250EA22EECF8D
:100ED00078F1EECF79F1EECF7AF1EECF7BF100EE43
:100EE00018F0E150E926E250EA22EECF7CF1EECF95
:100EF0007DF1EECF7EF1EECF7FF1110E806F816933
:100F0000826B836B8CDB67C1E1FF68C1E2FF00EE9F
:100F100014F0E150E926E250EA22EE2A000EEE2219
:100F2000EE22ED22ED52ED52050EE76E1200FFFFAC
:100F30008CD7FFFFD96E220D1C0EF324E16E000E3C
:100F4000F420E26E00EE0FF0E150E926E250EA22D2
:100F5000EF50006E0028D8B40AD000EE21F0E15026
:100F6000E926E250EA22EF50006E00B202D0000EF5
:100F7000CCD0010EE1240101726F000EE220736FEC
:100F800000EE0BF0E150E926E250EA22EECF74F1D8
:100F9000EDCF75F100EE0DF0E150E926E250EA22C6
:100FA000EECF76F1EDCF77F100EE14F0E150E926C7
:100FB000E250EA22EECF78F1EECF79F1EECF7AF17E
:100FC000EECF7BF100EE18F0E150E926E250EA2284
:100FD000EECF7CF1EECF7DF1EECF7EF1EECF7FF163
:100FE000100E806F00EE0FF0E150E926E250EA2289
:100FF000EF50816F00EE10F0E150E926E250EA2256
:10100000EECF82F1EDCF83F1E1CF70F1E2CF71F15C
:1010100006DB70C1E1FF71C1E2FF00EE14F0E150A8
:10102000E926E250EA22EECF18F0EECF19F0EECF2B
:101030001AF0EDCF1BF0ED52ED5200EE10F0E15042
:10104000E926E250EA22EECF00F0EDCF01F000C039
:1010500012F001C013F000EE10F0E150E926E2506A
:10106000EA22EECF00F0EDCF01F000EE14F0E150F7
:10107000E926E250EA220050EE260150EE22000E50
:10108000EE22ED22ED52ED5200EE14F0E150E92691
:10109000E250EA22EECF18F0EECF19F0EECF1AF0C0
:1010A000EDCF1BF0ED52ED5200EE21F0E150E926BC
:1010B000E250EA22FD0EEF1600EE21F0E150E926A3
:1010C000E250EA22EF0EEF16010100EE0FF0705130
:1010D000E9267151EA22EF50B7EC29F070C1E1FF27
:1010E00071C1E2FF00EE0FF0E150E926E250EA2282
:1010F000FF0EEF6E00EE21F0E150E926E250EA2209
:10110000EF50FD0B0209EF6E010E1200FFFF12D728
:10111000FFFFD96E220D2B0EF324E96E000EF42092
:10112000EA6EEF50006E0028D8A403D0EFEC28F050
:101130000AD0D950220D3D0EF324E96E000EF420A2
:10114000EA6EEF30010B1200FFFFE3D76A01FFFFE9
:10115000D96E220D1C0EF32401016E6F000EF420D7
:101160006F6FD9506B6F00EE0FF06E51E9266F5123
:10117000EA22EF50006E0028D8A426D000EE0FF02F
:101180006E51E9266F51EA2273C5EFFF00EE0FF0B2
:101190006E51E9266F51EA22EF50A9EC29F00101C6
:1011A00000EE10F06E51E9266F51EA22EE6AED6A08
:1011B000280EAA6FAB6B00EE0FF06E51E9266F514F
:1011C000EA22EF509BEC2BF0010100EE10F06E5183
:1011D000E9266F51EA22EECF6CF1EDCF6DF1030EEF
:1011E0006D5DCA0ED8B46C5DD8A002D0000E26D0BA
:1011F000010100EE21F06E51E9266F51EA22EF5015
:10120000EF0B1009EF6E6A51F6EC28F001016C2B20
:10121000000E6D2300EE10F06E51E9266F51EA22A8
:101220006CC1EEFF6DC1EDFF030E6D5DCA0ED8B44B
:101230006C5DD8A002D06B517CDE010E1200FFFF66
:1012400087D7FFFFD96E220D1C0EF324E16E000E2E
:10125000F420E26EE1CF69F1E2CF6AF100EE21F015
:10126000E150E926E250EA22EF50006E00B602D0CB
:10127000000E0CD0C7EC29F0010100EE21F06951FD
:10128000E9266A51EA22F70EEF16010E1200FFFF5F
:10129000D9D70001FFFFD96E220D1C0EF324E16E99
:1012A000000EF420E26E00EE21F0E150E926E2505B
:1012B000EA22EF50006E00A633D0E1CF00F1E2CF7A
:1012C00001F100EE21F0E150E926E250EA22EF5070
:1012D000006E00A40FD0280E01016A6F6B6B89ECC1
:1012E0002BF0010100EE21F00051E9260151EA2224
:1012F000FB0EEF16010100EE21F00051E92601512D
:10130000EA22EF50EF0B1009EF6E00C140F101C16E
:1013100041F102C142F103C143F171EC29F002D065
:10132000006A016A1200FFFFB6D76601FFFFD96E9F
:10133000220D1C0EF324E16E000EF420E26E00EE8E
:1013400021F0E150E926E250EA22EF50006E00A6BB
:1013500047D0E1CF68F1E2CF69F100EE21F0E15032
:10136000E926E250EA22EF50006E00A40FD0280ECA
:1013700001016A6F6B6B89EC2BF0010100EE21F02B
:101380006851E9266951EA22FB0EEF16010100EED1
:1013900012F06851E9266951EA22EE50ED10D8A406
:1013A0000CD0C7EC29F0010100EE21F06851E926CC
:1013B0006951EA22F70EEF1613D0010100EE12F088
:1013C0006851E9266951EA22EE06000EED5A5DECFD
:1013D00029F066C1E9FF67C1EAFFEF6E010E01D097
:1013E000000E1200FFFFA3D7FFFFD96E220D3D0EA6
:1013F000F324E96E000EF420EA6EEF30006E003246
:101400000030010B1200FFFFF0D7FFFF1200FFFFBB
:10141000FDD70601FFFF0101190E406F010E416F5C
:10142000140E426F436B71EC29F00101190EAA6F83
:10143000010EAB6F0FDB010100EE06F00651E9264D
:101440000751EA22EECF0DF1EECF0EF1EECF0FF104
:10145000EECF10F11EC211F11FC212F120C213F122
:1014600021C214F1156B060E166F08C117F109C1E0
:1014700018F117C1C5F118C1C6F135EC35F000C03F
:1014800017F101C018F101010D0EC36F010EC46FF9
:101490000C0EC56FC66B92EC35F0001C026E011C81
:1014A000036E02C00BF103C00CF1240E01016A6F40
:1014B0006B6B89EC2BF001010B51F6EC28F001016C
:1014C0000C51F6EC28F0140E01016A6F6B6B89EC7D
:1014D0002BF008C1AAF109C1ABF1A7D900C00BF1EB
:1014E00001C00CF101EE29F00101EE520C51ED1892
:1014F0000BC1E8FFD8B4EF18D8B403D0C7EC29F07B
:101500008AD0010125390F0B006ED8900036D89093
:101510000034EC0FD96E08C100F009C101F0005E83
:10152000000E015AEC0E0024086FFF0E0120096F17
:1015300025390F0B006E00C002F0036AD890023606
:101540000336D89002360336140E02246A6F000E5A
:1015500003206B6F89EC2BF00101190E2D6F010E2A
:101560002E6F06C12FF107C130F1A2D901010A6F18
:10157000FE0E0A610FD006C12DF107C12EF1190E22
:101580002F6F010E306F08C131F109C132F10A51DC
:1015900094DB41D0C7EC29F001010A29D8A43BD043
:1015A00008C100F009C101F0026A036A0050212756
:1015B00001502223025023230350242326B302D0B8
:1015C00026A106D00101212B000E22232323242350
:1015D00006C172F107C173F11BC174F11CC175F131
:1015E00019C176F11AC177F121C178F122C179F1DF
:1015F00023C17AF124C17BF11DC17CF11EC17DF1B3
:101600001FC17EF120C17FF1040E0101806F81694D
:10161000826B836B04D8010CFFFFFDD67201FFFFC4
:10162000EFEC28F00009D8B4FBD774C196F175C16E
:1016300097F176C198F177C199F178C19AF179C1A2
:101640009BF17AC19CF17BC19DF17CC19EF17DC172
:101650009FF17EC1A0F17FC1A1F101013F0EA3174F
:10166000F00EA2178051A36FDDEC29F000C0A4F1A9
:1016700001C0A5F101EEA4F0EE52040EED5C000EE7
:10168000D8B4EF5CD8A005D00101A46B040EA56FFF
:1016900012D001EEA4F0EE52000EED5C370ED8B47D
:1016A000EF5C0101D8A005D0CA0EA427FF0EA52328
:1016B00002D0A46BA56B0101A66BA76BA86BA96BED
:1016C000960EAA6F010EAB6FC5D9140E01018227C9
:1016D000000E832380A30ED0040E8227000E8323E6
:1016E000020E866F040E876F886F896BA2510F0BF5
:1016F000600904D00101A2510F0B5009A26F1EC254
:101700008AF11FC28BF120C28CF121C28DF101013F
:1017100000EE06F07251E9267351EA22EECF8EF107
:10172000EECF8FF1EECF90F1EECF91F1926B060EEE
:10173000936F82C194F183C195F194C1C5F195C1B4
:10174000C6F135EC35F000C094F101C095F101010E
:101750008A0EC36F010EC46F0C0EC56FC66B92EC80
:1017600035F0001C026E011C036E02C0A6F103C01E
:10177000A7F1A6C184F1A7C185F101018129D8B4DF
:1017800073C581F1140EAA6FAB6B81519BEC2BF0EA
:1017900072C1AAF173C1ABF1060E0101AC6F82C137
:1017A000ADF183C1AEF17CEC2FF00101960ECB6F51
:1017B000010ECC6F140ECD6FCE6B0EEC29F0010133
:1017C00080A309D0860ECB6F010ECC6F040ECD6FB7
:1017D000CE6B0EEC29F0140E0101AA6FAB6B815198
:1017E0009BEC2BF082C1AAF183C1ABF11ED800C0E3
:1017F00084F101C085F1240E0101AA6FAB6B815108
:101800009BEC2BF001018551F6EC28F0010184518D
:10181000F6EC28F00101AA6BAB6B81519BEC2BF02D
:1018200004EF2BF0FFFFFCD6AA01FFFF010E010120
:10183000AC6FAE6BAF6B0101AA51006EAB51016E84
:10184000AA07000EAB5B01500010D8B422D05DECAB
:1018500029F00101AD6FAC51D8A40AD0AD51AE252D
:10186000AE6FAD51AE610ED0AF3F0CD0AE2B0AD0F3
:101870000101AD51AF25AF6FAD51AF6103D0AE3FA8
:1018800001D0AF2B0101AC51000ED8B4010EAC6FEA
:10189000D2D70101AF51FF0AAF6FAE51FF0AAE6F51
:1018A000AEC100F0AFC101F01200FFFFBFD72D01A4
:1018B000FFFFFE0E0101316F016A0150220D1C0E67
:1018C000F324D96E000EF420DA6EDF50D8B44ED077
:1018D000010110EE02F02D51E1262E51E22200EE20
:1018E0000BF0D950E926DA50EA22EE52E652E550E2
:1018F000ED18E7CFE8FFD8B4EF18D8A437D0DF5001
:10190000006E0004D8A402D00150316F2DC1E9FF50
:101910002EC1EAFF10EE0DF0D950E126DA50E22296
:10192000E652EE52ED50E518EFCFE8FFD8B4E718D5
:10193000D8A41CD0010110EE06F02F51E126305141
:10194000E22200EE07F0D950E926DA50EA22EE5002
:10195000E61808E1EE50E61805E1EE50E61802E15F
:10196000EE50E618D8A402D0015070D0012A040E1F
:101970000164A3D701013151220D1C0EF324E16E45
:10198000000EF420E26E3151FE0AD8B457D0E75071
:10199000006E0004D8A452D0010EE124466F000E60
:1019A000E220476FE1CF32F1E2CF33F12FC148F1AE
:1019B00030C149F10A0E4A6F4B6B56EC38F032C118
:1019C000D9FF33C1DAFF010110EE02F02D51E126FB
:1019D0002E51E22200EE0BF0D950E926DA50EA222D
:1019E000E6CFEEFFE5CFEDFF2DC1E9FF2EC1EAFF07
:1019F00010EE0DF0D950E126DA50E222EECFE6FFEC
:101A0000EDCFE5FF00EE21F0D950E926DA50EA22C9
:101A1000F70EEF1600EE0FF0D950E926DA50EA2261
:101A2000FF0EEF6E00EE21F0D950E926DA50EA22DF
:101A3000EF50FD0B0209EF6E315108D00101315119
:101A4000FE0AD8A402D0FF0E01D0FE0E1200FFFF46
:101A500030D7AA01FFFFAAC1E9FFABC1EAFFEECF71
:101A6000C5F1EDCFC6F135EC35F0AAC1E9FFABC148
:101A7000EAFF00C0EEFF01C0EDFF010100EE02F041
:101A8000AA51E926AB51EA22EECFC5F1EDCFC6F15E
:101A900035EC35F0010100EE02F0AA51E926AB5118
:101AA000EA2200C0EEFF01C0EDFF00EE04F0AA51F3
:101AB000E926AB51EA22EECFACF1EECFADF1EECF9D
:101AC000AEF1EECFAFF149EC35F0010100EE04F0DC
:101AD000AA51E926AB51EA2200C0EEFF01C0EEFF99
:101AE00002C0EEFF03C0EEFF00EE08F0AA51E926A7
:101AF000AB51EA22EECFACF1EECFADF1EECFAEF1CD
:101B0000EECFAFF149EC35F0010100EE08F0AA513B
:101B1000E926AB51EA2200C0EEFF01C0EEFF02C091
:101B2000EEFF03C0EEFF00EE0EF0AA51E926AB5126
:101B3000EA22EECFC5F1EDCFC6F135EC35F001016B
:101B400000EE0EF0AA51E926AB51EA2200C0EEFFEA
:101B500001C0EDFF00EE10F0AA51E926AB51EA22D8
:101B6000EECFC5F1EDCFC6F135EC35F0010100EE59
:101B700010F0AA51E926AB51EA2200C0EEFF01C0E5
:101B8000EDFF00EE12F0AA51E926AB51EA22EECFAA
:101B9000C5F1EDCFC6F135EC35F0010100EE12F0E4
:101BA000AA51E926AB51EA2200C0EEFF01C0EDFFC9
:101BB0001200FFFF50D76901FFFF010100EE0FF097
:101BC0006951E9266A51EA22EF50006E0028D8B424
:101BD0001FD000EE0FF06951E9266A51EA22EF505A
:101BE000B7EC29F069C1E1FF6AC1E2FF00EE0FF036
:101BF000E150E926E250EA22FF0EEF6E00EE21F0FE
:101C0000E150E926E250EA22EF50FD0B0209EF6EA7
:101C100069C1E1FF6AC1E2FF00EE07F0E150E92689
:101C2000E250EA22EE6AEE6AEE6AED6A00EE0DF02C
:101C3000E150E926E250EA22EE6AED6AE1CF69F16D
:101C4000E2CF6AF100EE21F0E150E926E250EA220B
:101C5000EF50006E00B6C7EC29F069C1E1FF6AC120
:101C6000E2FF00EE21F0E150E926E250EA22F70E11
:101C7000EF1600EE1FF0E150E926E250EA22580E7E
:101C8000EE6E020EED6E00EE21F0E150E926E2501C
:101C9000EA22EF0EEF1600EE21F0E150E926E250C5
:101CA000EA22EF50006E00A002D0010E01D0000E1B
:101CB000E76E1200FFFF81D72D01FFFFD96E0101F2
:101CC000336BD950220D1C0EF324E16E000EF4206C
:101CD000E26E00EE18F0E150E926E250EA22EECF83
:101CE00036F1EECF37F1EECF38F1EECF39F100EE2D
:101CF00014F0E150E926E250EA22EECF3AF1EECFBD
:101D00003BF1EECF3CF1EECF3DF100EE04F02F5170
:101D1000E9263051EA22EECF42F1EECF43F1EECF89
:101D200044F1EECF45F131C100F032C101F0026A59
:101D3000036A0050422701504323025044230350BA
:101D4000452300EE14F0E150E926E250EA22EECFFE
:101D50003EF1EECF3FF1EECF40F1EECF41F100EE9C
:101D60001CF0E150E926E250EA22EF6AE1CF34F1BB
:101D7000E2CF35F1FBEC38F0010100EE1DF03451FB
:101D8000E9263551EA2200C0EEFF01C0EDFF34C163
:101D9000D9FF35C1DAFF00EE1FF0D950E926DA503D
:101DA000EA22580EEE6E020EED6EDF50006E000459
:101DB000D8A4A2D0C7EC29F034C1D9FF35C1DAFFCD
:101DC0000001142B000E15231623172300EE14F028
:101DD000D950E926DA50EA2214C0EEFF15C0EEFF12
:101DE00016C0EEFF17C0EEFF0101422B000E432389
:101DF0004423452300EE18F0D950E926DA50EA22B0
:101E000042C1EEFF43C1EEFF44C1EEFF45C1EEFF0C
:101E100000EE14F0D950E926DA50EA22EECF3EF176
:101E2000EECF3FF1EECF40F1EECF41F100EE14F0F6
:101E3000D950E926DA50EA22EE2A000EEE22EE22EE
:101E4000ED22ED52ED522FC1E1FF30C1E2FF00EE75
:101E50000DF0E150E926E250EA22EF50006E00A2B8
:101E600026D0010ED924466F000EDA20476F2DC10F
:101E700048F12EC149F10A0E4A6F4B6B56EC38F00F
:101E800034C1D9FF35C1DAFF2FC1E9FF30C1EAFF04
:101E900010EE0DF0D950E126DA50E222EECFE6FF47
:101EA000EDCFE5FF120E0101336F020E64D2040E76
:101EB0000101336F42C13EF143C13FF144C140F1E2
:101EC00045C141F100EE04F0E150E926E250EA227A
:101ED000EECF42F1EECF43F1EECF44F1EECF45F13C
:101EE00000EE07F0D950E926DA50EA22000EEE6E35
:101EF000EE6EEE6EED6E5AD22FC1E1FF30C1E2FF01
:101F000000EE0DF0E150E926E250EA22EF50006EBB
:101F100000A408D0C7EC29F034C169F135C16AF1D9
:101F20004BDE75D200EE08F0E150E926E250EA22DD
:101F30000101EE503E1908E1EE503F1905E1EE5067
:101F4000401902E1EE504119D8A42ED2DF50020A06
:101F5000D8A456D000EE0DF0E150E926E250EA2276
:101F6000EF50006E00A849D000EE18F0D950E926D5
:101F7000DA50EA2242C1EEFF43C1EEFF44C1EEFF58
:101F800045C1EEFF00EE1CF0D950E926DA50EA22F6
:101F9000EF6AFBEC38F0010100EE1DF03451E92648
:101FA0003551EA2200C0EEFF01C0EDFF34C1E1FF70
:101FB00035C1E2FF040EE76E32513111D8B41AD0A8
:101FC00000EE21F0E150E926E250EA22EF50F70B53
:101FD0000809EF6E00EE12F0E150E926E250EA2225
:101FE00031C1EEFF32C1EDFF00EE21F0E150E926F4
:101FF000E2506DD0C7EC29F0D9D1C7EC29F0D6D189
:10200000DF50030AD8A46FD000EE0DF0E150E926AE
:10201000E250EA22EF50006E00A262D00101422B92
:10202000000E43234423452300EE18F0D950E9263F
:10203000DA50EA2242C1EEFF43C1EEFF44C1EEFF97
:1020400045C1EEFF00EE0DF0E150E926E250EA2234
:10205000EF50006E00A805D0100E336F040EDF6E37
:1020600018D0120E0101336F020EDF6E3E2B000EF0
:102070003F234023412300EE14F0D950E926DA50E3
:10208000EA223EC1EEFF3FC1EEFF40C1EEFF41C17B
:10209000EEFF010132513111D8B41FD000EE21F012
:1020A000D950E926DA50EA22EF50F70B0809EF6E13
:1020B00000EE12F0D950E926DA50EA2231C1EEFFE3
:1020C00032C1EDFF00EE21F0D950E926DA50EA22C4
:1020D000EF50FB0B0409EF6E69D1C7EC29F066D114
:1020E000C7EC29F063D110EE18F0D950E126DA5090
:1020F000E222010100EE04F02F51E9263051EA22DC
:10210000EE50E61808E1EE50E61805E1EE50E6184C
:1021100002E1EE50E618D8B403D0C7EC29F077D12D
:1021200000EE18F0D950E926DA50EA2242C1EEFF5B
:1021300043C1EEFF44C1EEFF45C1EEFFDF50040A8C
:10214000D8A4BFD0010100EE0DF02F51E926305187
:10215000EA22EF50006E00A82AD000EE0FF0D9500E
:10216000E926DA50EA22EF50006E0028D8B41FD0DA
:1021700000EE0FF03451E9263551EA22EF50B7EC6A
:1021800029F034C1D9FF35C1DAFF00EE0FF0D95084
:10219000E926DA50EA22FF0EEF6E00EE21F0D95068
:1021A000E926DA50EA22EF50FD0B0209EF6E010139
:1021B00000EE0DF02F51E9263051EA22EF50006E6B
:1021C00000A02BD0110E336F00EE14F0D950E92689
:1021D000DA50EA223FEC39F000C03EF101C03FF195
:1021E00002C040F103C041F100EE18F0D950E926D9
:1021F000DA50EA22EE2A000EEE22EE22ED22ED5215
:10220000ED52EECF42F1EECF43F1EECF44F1EDCF00
:1022100045F1ED52ED520A0EDF6E010132513111DE
:10222000D8B44CD000EE21F0D950E926DA50EA2299
:10223000EF50006E00B621D000EE21F0D950E92613
:10224000DA50EA22EF50F70B0809EF6E00EE12F0B9
:10225000D950E926DA50EA2231C1EEFF32C1EDFF52
:1022600000EE21F0D950E926DA50EA22EF50FB0BBC
:102270000409EF6E100E336F99D00101336B00EE3D
:1022800014F0D950E926DA50EA223AC1EEFF3BC1F8
:10229000EEFF3CC1EEFF3DC1EEFF00EE18F0D9505D
:1022A000E926DA50EA2236C1EEFF37C1EEFF38C127
:1022B000EEFF39C1EEFFC7EC29F078D0C7EC29F06A
:1022C00075D0DF500A0AD8A413D0C7EC29F0010159
:1022D00000EE0DF02F51E9263051EA22EF50006E4A
:1022E00000A864D034C169F135C16AF165DC5ED003
:1022F000DF50050AD8A441D0C7EC29F02FC1E1FF77
:1023000030C1E2FF00EE0DF0E150E926E250EA2292
:10231000EF50006E00A04AD0100E0101336F34C19F
:10232000D9FF35C1DAFF00EE18F0D950E926DA50AE
:10233000EA22EE2A000EEE22EE22ED22ED52ED52BE
:10234000EECF42F1EECF43F1EECF44F1EDCF45F1C8
:10235000ED52ED5200EE0DF0E150E926E250EA2296
:10236000EF50006E00A806D0D9CF69F1DACF6AF13C
:1023700023DC1CD0060EDF6E19D0DF50060AD8A46D
:1023800015D0C7EC29F0010100EE0DF02F51E92620
:102390003051EA22EF50006E00A808D034C169F134
:1023A00035C16AF109DC02D0C7EC29F001013351D3
:1023B000D8B42DD02DC172F12EC173F12FC1E1FF20
:1023C00030C1E2FF00EE02F0E150E926E250EA22DD
:1023D000EECF74F1EDCF75F1E6CF76F1E5CF77F181
:1023E0003EC178F13FC179F140C17AF141C17BF141
:1023F00042C17CF143C17DF144C17EF145C17FF111
:102400003351806F8169826B836B0FEC0BF012008C
:10241000FFFF54D4FFFF42D005EC39F0E2C5F3FFD3
:10242000E3C5F4FFE4C5F5FFE5C5F6FFE6C5F7FF34
:10243000E7C5F8FFE8C500F0E9C501F0EAC502F01C
:10244000EBC503F0ECC504F0EDC505F0EEC506F0F4
:10245000EFC507F0F0C508F0F1C509F0F2C50AF0C4
:10246000F3C50BF0F4C50CF0F5C50DF0F6C50EF094
:10247000F7C5DAFFF8C5D9FFF9C5E2FFFAC5E1FFF4
:10248000FBC5EAFFFCC5E9FFFDC5E8FFFEC5FAFF95
:10249000FFC5D8FF0FC0E0FF1000FFFFBDD7E0CFA2
:1024A0000FF0E8CFFDF5E9CFFCF5EACFFBF5E1CF82
:1024B000FAF5E2CFF9F5D9CFF8F5DACFF7F50EC096
:1024C000F6F50DC0F5F50CC0F4F50BC0F3F50AC038
:1024D000F2F509C0F1F508C0F0F507C0EFF506C048
:1024E000EEF505C0EDF504C0ECF503C0EBF502C058
:1024F000EAF501C0E9F500C0E8F5F8CFE7F5F7CF58
:10250000E6F5F6CFE5F5F5CFE4F5F4CFE3F5F3CF57
:10251000E2F580D7FFFF0CD00101A96F00D0ACA27B
:1025200001D001D0FCD70101A951AD6E1200FFFF0F
:10253000F3D72B01FFFF14D003D001012D51EADFA7
:102540002BC1E9FF2CC1EAFF01012B4B2C2BEF50D3
:102550002D6F2D51D8A401D001D0EFD71200FFFF6D
:10256000EBD7FFFF42D0F86AF6DAEDEC38F0E1EC99
:1025700032F00FDB81BA01D001D002D029EC18F083
:1025800094EC31F028EC19F091EC24F036C200F014
:1025900000A001D001D001D006D0010EE8CF9AF5FD
:1025A000070EE8CF6FF50101640E2B6F050E2C6F3F
:1025B000C1DF18D0A3EC31F04DEC19F0A9EC24F0F8
:1025C000D9D8DFC5E8FF05019A19D8B401D001D0E8
:1025D00009D001011E0E1E6F020E1F6F206B07D85F
:1025E000DFC59AF5E7D70CEF00F0BDD71E01FFFF5E
:1025F000C0D001012051D8B401D001D000D00101D8
:10260000210E2D6F010E2E6F4F0E2F6F090E306FA2
:102610001EC1E9FF1FC1EAFFEF50006E00C002F0CB
:10262000036A02C029F103C02AF1290EE8CF2BF179
:10263000010EE8CF2CF1B9EC2BF001012051D8B4F8
:1026400001D001D001D008D00101210E2B6F010E65
:102650002C6F70DF2E0E5EDF0101210E2D6F010E3B
:102660002E6F4F0E2F6F090E306F00EE01F01E51CE
:10267000E9261F51EA22EF50006E00C002F0036A03
:1026800002C029F103C02AF1290EE8CF2BF1010E77
:10269000E8CF2CF1B9EC2BF001012051D8B401D0D6
:1026A00001D001D008D00101210E2B6F010E2C6F3B
:1026B00041DF2E0E2FDF0101210E2D6F010E2E6F37
:1026C0004F0E2F6F090E306F00EE02F01E51E926FB
:1026D0001F51EA22EF50006E00C002F0036A02C0F0
:1026E00029F103C02AF1290EE8CF2BF1010EE8CF22
:1026F0002CF1B9EC2BF001012051D8B401D001D05C
:1027000001D008D00101210E2B6F010E2C6F12DFBA
:102710002E0E00DF0101210E2D6F010E2E6F4F0EC8
:102720002F6F090E306F00EE03F01E51E9261F5186
:10273000EA22EF50006E00C002F0036A02C029F1E5
:1027400003C02AF1290EE8CF2BF1010EE8CF2CF1BE
:10275000B9EC2BF001012051D8B401D001D001D047
:1027600006D00101210E2B6F010E2C6FE3DE12004B
:10277000FFFF3FD7FFFF5ED0810EC26E640E0101E6
:10278000006F00D0010100070029D8A401D001D0BA
:10279000F9D7C28400D0C2B401D001D0FCD7C35055
:1027A0000101006FC450016F9B0E2D6F050E2E6F3F
:1027B0004F0E2F6F090E306F00C102F101C103F1FE
:1027C000020EE8CF2BF1010EE8CF2CF1B9EC2BF083
:1027D000840EC16E890EC26E640E0101006F00D0BE
:1027E000010100070029D8A401D001D0F9D7C28483
:1027F00000D0C2B401D001D0FCD7C3500101006F9A
:10280000C450016FA30E2D6F050E2E6F4F0E2F6F4C
:10281000090E306F00C102F101C103F1020EE8CFD1
:102820002BF1010EE8CF2CF1B9EC2BF08E0EC16E1E
:102830001200FFFFA1D76601FFFF67D066C1E9FF65
:1028400067C1EAFFEECF00F0EDCF01F000C0E9FF75
:1028500001C0EAFFEF50D00F0101696F4DD00101B7
:1028600000EE02F06651E9266751EA22EECF00F051
:10287000EDCF01F000C0E9FF01C0EAFFEF50D00F3B
:102880006A6F09D0897612D0897410D08B700ED0FF
:102890008B720CD00BD001016A51000AF3E0010ADF
:1028A000F3E0090AF3E0010AF3E000D066C1E9FFB2
:1028B00067C1EAFFEECF76F1EDCF77F101018F0E20
:1028C000786F070E796F0D0E7A6F12EC36F01BD011
:1028D0001AD066C1E9FF67C1EAFFEECF76F1EDCF0E
:1028E00077F101019C0E786F070E796F0A0E7A6FEF
:1028F00012EC36F008D007D001016951000AAFE0B0
:10290000010AE6E0E6D71200FFFF98D76A01FFFF51
:10291000EFD001016E6FCDD089A601D001D007D0D4
:102920006CC1E9FF6DC1EAFF300EEF6E06D06CC1DD
:10293000E9FF6DC1EAFF310EEF6ED3D089A401D05B
:1029400001D007D06CC1E9FF6DC1EAFF300EEF6E18
:1029500006D06CC1E9FF6DC1EAFF310EEF6EC1D048
:102960008BA001D001D007D06CC1E9FF6DC1EAFF97
:10297000300EEF6E06D06CC1E9FF6DC1EAFF310E7B
:10298000EF6EAFD08BA201D001D007D06CC1E9FFB0
:102990006DC1EAFF300EEF6E06D06CC1E9FF6DC16C
:1029A000EAFF310EEF6E9DD001016B516A11D8A480
:1029B00001D001D002D06A6B6B6B01016A5115EE38
:1029C0009BF0E126000EE2226CC1E9FF6DC1EAFF37
:1029D000E7CFEFFF6A5105EE9BF0E926000EEA22F1
:1029E000EF50D8A401D001D005D0FF0E006EFF0E2D
:1029F000016E7CD0010E01016A27000E6B236AC1B3
:102A000000F06BC101F072D001016B516A11D8A4C2
:102A100001D001D002D06A6B6B6B01016A5115EED7
:102A2000A3F0E126000EE2226CC1E9FF6DC1EAFFCE
:102A3000E7CFEFFF6A5105EEA3F0E926000EEA2288
:102A4000EF50D8A401D001D005D0FF0E006EFF0ECC
:102A5000016E4CD0010E01016A27000E6B236AC182
:102A600000F06BC101F042D081AA01D001D007D0A3
:102A70006CC1E9FF6DC1EAFF310EEF6E06D06CC18B
:102A8000E9FF6DC1EAFF300EEF6E2BD082A401D0BA
:102A900001D007D06CC1E9FF6DC1EAFF310EEF6EC6
:102AA00006D06CC1E9FF6DC1EAFF300EEF6E19D0A0
:102AB00018D001016E51000A01E12ED7010A01E18F
:102AC0003DD7030A01E170D7010A9EE0070ACCE076
:102AD000020ADCE00E0A01E143D7010A01E152D704
:102AE00000D0FF0E006EFF0E016E00D01200FFFF3F
:102AF00010D70601FFFF2ED006C176F107C177F18E
:102B00000101A60E786F070E796F030E7A6F7B6B4B
:102B100091EC1FF001500010D8A401D001D016D0C4
:102B200008C176F109C177F10101AA0E786F070E8D
:102B3000796F030E7A6F7B6B91EC1FF001500010E0
:102B4000D8A401D001D002D0010E02D0000E00D0D6
:102B50001200FFFFD1D7FFFF1BD08E0EC16E030EF8
:102B6000926E809A89848986F19E82908292829464
:102B70009480948294848B808B82200EAC6E900E15
:102B8000AB6E0F0EAF6ED56AF28EF28C1200FFFFA5
:102B9000E4D7FFFF6CD00A0EE8CF1EF20A0EE8CF92
:102BA0001FF2050EE8CF20F20F0EE8CF21F2FF0E44
:102BB000E8CF28F2FF0EE8CF29F2FF0EE8CF2AF285
:102BC00002012B6B0A0EE8CF2CF20A0EE8CF2DF291
:102BD000050EE8CF2EF20F0EE8CF2FF2226B040E77
:102BE000E8CF23F2A30EE8CF24F2256B266B276BE8
:102BF000368101011E0E016F020E026F816B826B26
:102C0000A00E54EC1EF0E3EC1EF00101006FEFEC9F
:102C10001EF001010051550AD8A401D001D024D0E2
:102C2000010E816F826BA00E54EC1EF00101006B4F
:102C3000180E006501D001D001D013D0E3EC1EF0D6
:102C400001C1E9FF02C1EAFFEF6E010E0101012798
:102C5000000E0223010E0027180E006501D001D0DE
:102C6000EDD7EFEC1EF001D003D81200FFFF93D791
:102C7000FFFF2BD001011E0E1F6F020E206FAB6BEA
:102C8000AC6BA00EEDEC1DF0550E9CEC1EF001019E
:102C90001E6B180E1E6501D001D001D012D01FC1CD
:102CA000E9FF20C1EAFF01011F4B202BEF509CECF4
:102CB0001EF0010E01011E27180E1E6501D001D065
:102CC000EED7CDEC1EF01200FFFFD4D71E01FFFFA0
:102CD00021D003D0010120511DDC01011EC1F6FFEE
:102CE0001FC1F7FF010E1E27000E1F23050EF764FC
:102CF00004D00800FFFFF55005D0F6CFE9FFF7CF6D
:102D0000EAFFEF50206F2051D8A401D001D0E2D7C4
:102D10001200FFFFDED71E01FFFF38D00101226B3A
:102D200000D09EAA01D001D0FCD7AE500101216F86
:102D300021510D0AD8A401D005D021510A0AD8A4E6
:102D400002D000D002D000D001D01BD0010E010172
:102D500022271EC1E9FF1FC1EAFF21C1EFFF010EBB
:102D60001E27000E1F231EC1E9FF1FC1EAFF000E30
:102D7000EF6E20072029D8A401D001D001D001D0C6
:102D8000CFD70101225100D01200FFFFC7D71E018B
:102D9000FFFF64D01EC123F11FC124F10101256B87
:102DA0003AD0010122512E0AD8A401D001D020D05E
:102DB0001EC1E9FF1FC1EAFF000EEF6E010E1E27C4
:102DC000000E1F2323C126F124C127F1F0EC36F0B9
:102DD000010125512025E96E000E2121EA6E00C077
:102DE000EFFF010E25271EC123F11FC124F10ED0D4
:102DF000300E0101226101D004D0390E226502D0CB
:102E000000D002D000D002D0000E26D0010E010169
:102E10001E27000E1F231EC1E9FF1FC1EAFFEF504E
:102E20000101226F2251D8A401D001D0BAD723C109
:102E300026F124C127F1F0EC36F0010125512025BF
:102E4000E96E000E2121EA6E00C0EFFF2551030A52
:102E5000000ED8B4010E00D01200FFFF9BD7FFFF79
:102E60001BD000D09EAA01D001D0FCD7AE500101EA
:102E7000016F300E016506D000D0390E016102D01D
:102E800000D002D000D004D00101015103D002D003
:102E9000390E00D01200FFFFE4D7FFFFD9D00101A7
:102EA0001B6F0D0E8AEC12F00A0E8AEC12F0010173
:102EB0001B51020D6C0EF324E96E000EF420EA6E35
:102EC000EECF1EF1EDCF1FF102DFACD00101010EFC
:102ED0002D6F010E2E6F4F0E2F6F090E306F02EE09
:102EE00030F0EECF1CF1EDCF1DF11C0EE8CF2BF131
:102EF000010EE8CF2CF1B9EC2BF00101010E2B6F84
:102F0000010E2C6F9AEC12F0290E8AEC12F03A0E98
:102F10008AEC12F0200E8AEC12F00101010E1E6FF5
:102F2000010E1F6F140E206FF7DE006E00C002F05E
:102F3000036A03500210D8B401D001D00FD0010EA3
:102F4000266F010E276FF0EC36F000C030F201C0A2
:102F500031F231C226F230C227F201D03ED076D013
:102F600001011E0E196F020E1A6F0BD001012C0EFB
:102F7000196F020E1A6F05D00101280E196F020E8B
:102F80001A6F19C11EF11AC11FF10101206BF7EC74
:102F900012F0290E8AEC12F03A0E8AEC12F0200E92
:102FA0008AEC12F00101010E1E6F010E1F6F140E4C
:102FB000206FB2DE010E1E6F010E1F6F150E206F07
:102FC000010E216FE5DE006E00C002F0036A0350BF
:102FD0000210D8A401D001D00DD00101050E1E6F42
:102FE000090E1F6F74DE00D09EAA01D001D0FCD75D
:102FF000AE500CD019C1E9FF1AC1EAFF15C1EEFFAE
:1030000016C1EEFF17C1EEFF18C1EEFF1FD002017F
:1030100036811CD00201369119D038D817D028DE5D
:1030200015D014D001011B51310A01E14FD7030A19
:1030300097E0010A9BE0070A9FE0010AE8E0030A23
:10304000E9E0010AEAE00F0AEAE000D01200FFFF1F
:1030500026D7FFFF1AD00101AE0E1E6F070E1F6F9D
:1030600036DEFDDE0101006F0051390AD8B401D00F
:1030700001D002D0005111DF01010051380AD8A45B
:1030800001D001D0E8D71200FFFFE5D7FFFFDFD066
:1030900001011E6B226BBCEC33F000C020F101C0BB
:1030A00021F1FBEC38F000C0A5F101C0A6F105EC60
:1030B00039F0FBEC38F000C0A7F101C0A8F1010124
:1030C000A651A85D02E1A551A75DD8A021D000D0EE
:1030D000A7C100F0A8C101F0A551005EA651015A98
:1030E000000E015C050ED8B4005C000ED8B0010ED5
:1030F000006E016A0ED0FF0E006EFF0E016EA5512C
:10310000005EA651015AA7510026A851012201D004
:10311000F2D701500010D8B401D001D00AD0FBEC96
:1031200038F000C0A5F101C0A6F1150E8AEC12F02E
:1031300089749EAA01D001D0BAD77FD005EC39F0AE
:103140009EAA01D001D005D08974AE5001011F6F35
:1031500001D073D069D001011F05D8A401D001D0DE
:1031600003D0010E1E6F14D001011F51040AD8A410
:1031700001D001D00AD0898465EC33F0060E8AECC8
:1031800012F0010E0101226F03D0150E8AEC12F02D
:1031900054D0060E0101246F236B020E1E6F4DD01A
:1031A000030E01011E6F49D00101235101EE25F0EC
:1031B000E926000EEA221FC1EFFF010E2327800E31
:1031C000236501D001D02ED020C1A9F121C1AAF1DF
:1031D000C6EC33F0060E0101246F1F6B7F0E1F65D6
:1031E00001D001D001D012D001011F5101EE25F014
:1031F000E926000EEA22EF50E3EC33F0010E010164
:103200001F277F0E1F6501D001D0EED703EC34F0ED
:1032100000C020F101C021F1010124518AEC12F01B
:1032200001011E6B0AD009D001011E51010AB1E053
:10323000030AB6E0010AB8E08ED701012251D8B4E2
:1032400001D001D07BD7010E00D01200FFFF20D7A4
:10325000FFFF0101006B500E0101016F026BE6ECF4
:1032600005F0006E010100510A0D000EF324E96E15
:10327000020EF420EA6E00C0EFFF00510A0D030EAB
:10328000F324E96E020EF420EA6EEF6A002B020EC0
:103290000065E1D71200FFFFDCD7FFFF0101006BE3
:1032A0000101005108D80101002B020E0065F8D77A
:1032B0001200FFFFF3D7FFFFD96E0A0D000EF324B3
:1032C0000101096F020EF4200A6F010E026F0CD289
:1032D00009C1E9FF0AC1EAFFEF50F4EC09F0000967
:1032E000D8B402D2010E0101026F056B066B010119
:1032F000000E065D500ED8B4055DD8B01BD0055148
:10330000006E0651016E054B062B150E0024666FEC
:10331000010E0120676F09C1E9FF0AC1EAFFEF5002
:1033200096EC09F0006E00C002F0036A0350021030
:10333000D8A4DDD7010101EE15F00551E9260651AB
:10334000EA22EF6A09C1E9FF0AC1EAFFEF5021EC66
:1033500009F0010100EE03F00951E9260A51EA22C1
:10336000020EEF6E050E036F150E666F010E676F8E
:103370000B0E686F010E696F030E6A6F010E6B6FA3
:10338000090E09256C6F000E0A216D6FDADA010152
:10339000016F0151D8A4A8D1010E036511D00B0E05
:1033A000666F010E676F0351686F1CEC14F001012A
:1033B00000EE09F00951E9260A51EA22030EEF6EE8
:1033C0000BC166F10CC167F1EDEC32F0010100EECA
:1033D00001F00951E9260A51EA2200C0EEFF01C0BE
:1033E000EDFF09C1E1FF0AC1E2FF00EE01F0E1508B
:1033F000E926E250EA22EE52ED50FF0AFF0ED8B461
:10340000EF18D8A411D000EE08F0E150E926E25000
:10341000EA22000EEF6E00EE03F0E150E926E250E2
:10342000EA22020EEF6E60D100EE01F0E150E926D3
:10343000E250EA22EE50ED10D8A408D000EE08F0D9
:10344000E150E926E250EA22030EE4D700EE03F051
:10345000E150E926E250EA220B0EE4D709C1E9FF68
:103460000AC1EAFFEF5088EC08F000090101D8B466
:103470003CD100EE08F00951E9260A51EA22EF504A
:10348000020DC60EF324E96E000EF420EA6EEECFB4
:1034900007F1EDCF08F1010107C1F6FF08C1F7FF01
:1034A000072B000E0823050EF76404D00800FFFF69
:1034B000F55005D0F6CFE9FFF7CFEAFFEF50D96E10
:1034C000D950D8B40AD001016A6F09C1E9FF0AC115
:1034D000EAFFEF50A7EC08F0DED709C1E9FF0AC107
:1034E000EAFFEF5099EC07F0C1D009C1E9FF0AC12A
:1034F000EAFFEF5088EC08F00009D8B4F5D0010ECF
:103500000101026F046B04C100F0016A0050A80FB2
:10351000F66E0150F76E060EF7220800FFFFF55019
:1035200001016A6F09C1E9FF0AC1EAFFEF50A7EC88
:1035300008F00101042B1E0E0465E5D700EE09F02A
:103540000951E9260A51EA22EF50140D1C0EF3240A
:10355000076F060EF420086F010107C1F6FF08C1CE
:10356000F7FF072B000E0823050EF76404D00800B0
:10357000FFFFF55005D0F6CFE9FFF7CFEAFFEF5098
:10358000D96ED9500101D8B409D06A6F09C1E9FFD9
:103590000AC1EAFFEF50A7EC08F0DED7046B04C1C4
:1035A00000F0016A0050C80FF66E0150F76E060E6B
:1035B000F7220800FFFFF55001016A6F09C1E9FF1A
:1035C0000AC1EAFFEF50A7EC08F00101042B030E3B
:1035D0000465E5D709C1E1FF0AC1E2FF00EE09F089
:1035E000E150E926E250EA22EF50030A00EE07F02C
:1035F000D8A406D0E150E926E250EA22010E05D017
:10360000E150E926E250EA22000EEF6E00EE04F0EF
:10361000E150E926E250EA22030EEF6E00EE03F0DD
:10362000E150E926E250EA22010EFCD609C1E9FF89
:103630000AC1EAFFEF50F4EC09F00009D8B407D052
:1036400009C1E9FF0AC1EAFFEF5021EC09F009C105
:1036500066F10AC167F165D8006E00C002F0036A26
:1036600003500210D8B440D065EC33F0010100EEF5
:1036700003F00951E9260A51EA22090ED3D609C1FD
:10368000E9FF0AC1EAFFEF5013EC07F00009D8B4D4
:103690002BD009C1E9FF0AC1EAFFEF5088EC08F01E
:1036A0000009D8B421D009C1E9FF0AC1EAFFEF50EF
:1036B00024EC07F0010100EE03F00951E9260A515C
:1036C000EA220A0EAFD60951E9260A51EA22EF5042
:1036D00001E1FED5010AAAE0030A01E1BFD60B0A07
:1036E000CEE0020A01E101D701010251D8B415D0A0
:1036F0000101026B09C1E9FF0AC1EAFFEF5013ECB7
:1037000007F00009010100EE03F0D8A4DCD709514D
:10371000E9260A51EA22000EEF6A1200FFFFCCD51B
:103720006601FFFF010100EE01F06651E9266751D5
:10373000EA22EECF6AF1EDCF6BF174EC33F066C1A3
:10374000E9FF67C1EAFFEF5088EC08F00009D8B440
:10375000E6D00101686B00EE04F06651E92667517E
:10376000EA22EF50080AD8B417D08CEC33F00101EC
:10377000696F0101FD51FF0AFF0ED8B4FC19D8A4EE
:103780000BD0B2EC33F066C1E9FF67C1EAFFEF503E
:1037900099EC07F0010ED1D066C1E1FF67C1E2FFED
:1037A00000EE07F0E150E926E250EA22EF50D8A4FB
:1037B0008BD0AAD001016951250AD8A408D000EE07
:1037C00004F0E150E926E250EA22050E12D0010E83
:1037D0000101686F8BD001016951250AD8A40BD073
:1037E000010E686F00EE04F0E150E926E250EA2293
:1037F000030EEF6E7BD000EE08F0E150E926E250B8
:10380000EA2201016939F00BEF6E00EE04F0E1509D
:10381000E926E250EA22060EECD769C100F0D00E8C
:10382000002600EE08F0E150E926E250EA220050BE
:10383000EF1200EE04F0E150E926E250EA22080E11
:10384000EF6E00EE05F0E150E926E250EA22000EAC
:10385000EE6EED6E4BD0010100EE05F06651E926EB
:103860006751EA22EECF6AF1EDCF6BF1690E6C6F12
:10387000010E6D6F00EE08F06651E9266751EA22ED
:10388000EF5087EC14F0010100EE05F06651E926D7
:103890006751EA2200C0EEFF01C0EDFF010E686F24
:1038A00066C1E1FF67C1E2FF00EE05F0E150E926E5
:1038B000E250EA22EE52ED50FF0AFF0ED8B4EF18A4
:1038C000D8A414D08FD7FFD700EE04F0E150E9263A
:1038D000E250EA22EF50030A01E16CD7060A01E147
:1038E0007AD7030A9AE00E0AB6E0EDD701016851D3
:1038F000D8B425D769516A6F66C1E9FF67C1EAFF8D
:10390000EF50A7EC08F01BD7010169516A6F66C13F
:10391000E9FF67C1EAFFEF50A7EC08F010D7B2EC5F
:1039200033F0010100EE01F06651E9266751EA2209
:1039300000C0EEFF01C0EDFF000E1200FFFFF2D647
:103940006601FFFF01016F6B746B756B706B66C175
:1039500076F167C177F1CD0E786F060E796F030EA1
:103960007A6F7B6B91EC1FF001500010D8A40BD044
:1039700066C1E1FF67C1E2FF040EE126000EE2220C
:1039800001016E6B03D0020E14D1E652E750200AFB
:10399000D8B4FBD78ED06AC1E9FF6BC1EAFFEF5004
:1039A0000101705DD8B094D078D00101D890703505
:1039B000006E016A0136D9500024E96EDA50012008
:1039C000EA6EE1CFEEFFE2CFEDFFE750F36E2F0A94
:1039D000D8B422D0F3505C0AD8A46AD01DD001011B
:1039E000D8907035006E016A0136D9500024E96E16
:1039F000DA500120EA6EE1CFEEFFE2CFEDFF702B4F
:103A0000020E6F6FE750F36E3F0AD8B404D0F35044
:103A1000260AD8A405D0E76A010E01016F6F48D0CD
:103A2000F3502B0AD8A403D0200EE76E41D0F350F8
:103A30002E0AD8A40AD001017005D8A406D0E652F7
:103A4000E1CF74F1E2CF75F133D0F3503D0AD8B431
:103A5000E2D7F3502F0AD8B404D0F3505C0AD8A4AC
:103A600027D0E1CF00F0E2CF01F0002A000E0122C2
:103A70000101D8907035026E036A0336D9500226D0
:103A8000DA500322FE0E0224E96EFF0E0320EA6ED6
:103A900000C0EEFF01C0EDFF0BD068C1D9FF69C1C6
:103AA000DAFF01016F5181E0010A99E0030AAAE0FF
:103AB000E652E750D96E200AD8B40AD0D950D8B40B
:103AC00007D00D0AD8B404D0D9500A0AD8A463D7B5
:103AD000E76A6CC1E9FF6DC1EAFF070EEF6E0101F5
:103AE00075517411D8B432D074C17AF175C17BF1BB
:103AF000F6EC35F000C074F101C075F10101000E63
:103B0000726F060E736F716B74C176F175C177F1C8
:103B100072C178F173C179F1030E01017A6F7B6B89
:103B200091EC1FF001500010D8A407D06CC1E9FF40
:103B30006DC1EAFF71C1EFFF09D0040E01017227C8
:103B4000000E7323712B060E7165DED701017051D3
:103B5000D8A427D068C1E9FF69C1EAFFEECF76F1AA
:103B6000EDCF77F1D10E786F060E796F090E7A6F6F
:103B700012EC36F068C1E9FF69C1EAFFEECF00F050
:103B8000EDCF01F0090E0024E96E000E0120EA6E6F
:103B9000EF6A6CC1E9FF6DC1EAFF010EEF6E010132
:103BA000702B6AC1E9FF6BC1EAFF70C1EFFF010131
:103BB0006E511200FFFFC6D6FFFFD96E3F0EC7162B
:103BC000C66AC56AC686C75094869488C68AD95084
:103BD000C86E1200FFFFF1D7AB01FFFF0101AD6F0F
:103BE000ABC1AEF1ACC1AFF1C5CF00F01F0E0016F6
:103BF00000C002F0036A000EC7B4010E02120350A7
:103C00000210D8A4F1D7C580C5B0FED7A1B632D076
:103C10000101AD5171D90009D8A42CD0C5CF00F055
:103C20001F0E001600C002F0036A000EC7B4010E9A
:103C3000021203500210D8A4F1D7C5BC30D0010144
:103C4000AF515AD90009D8A415D0C5CF00F01F0E26
:103C5000001600C002F0036A000EC7B4010E021283
:103C600003500210D8A4F1D70101AE5145D9000983
:103C7000D8B402D0010E14D0C5CF00F01F0E00162C
:103C800000C002F0036A000EC7B4010E0212035016
:103C90000210D8A4F1D7C5BC02D0000E01D0020E8C
:103CA0001200FFFF9BD78101FFFF0101836F81C1DC
:103CB000ABF182C1ACF191DF0101846F8451D8A4D2
:103CC00006D0C0D80101846F8451D8B402D0845189
:103CD00030D0C5CF00F01F0E001600C002F0036AFE
:103CE000000EC7B4010E021203500210D8A4F1D77F
:103CF000C580C5B0FED7A1B606D001018329FCD886
:103D00000009D8B402D0010E14D0C5CF00F01F0EA8
:103D1000001600C002F0036A000EC7B4010E0212C2
:103D200003500210D8A4F1D7C5BC02D0000E01D0B8
:103D3000020E1200FFFFB9D7FFFF0101AA6FC5CF26
:103D400000F01F0E001600C002F0036A000EC7B498
:103D5000010E021203500210D8A4F1D70101AA519A
:103D6000CBD80009D8B402D0010E14D0C5CF00F0D2
:103D70001F0E001600C002F0036A000EC7B4010E49
:103D8000021203500210D8A4F1D7C5BC02D0000E15
:103D900001D0020E1200FFFFD0D7FFFFC5CF00F009
:103DA0001F0E001600C002F0036A000EC7B4010E19
:103DB000021203500210D8A4F1D7C584C5A4000C88
:103DC000FDD7FFFFEBD7FFFFA3D8C5B6FED7C59A37
:103DD000C588C5B8FED7C9501200FFFFF5D7FFFF51
:103DE00097D8C5B6FED7C58AC588C5B8FED7C584DD
:103DF000C5A4000CFDD7FFFFF3D77A01FFFF010137
:103E00007F6F7AC181F17BC182F14EDF0101806F4A
:103E10008051D8B40BD012D0D6DF7CC1E9FF7DC170
:103E2000EAFFEF6E01017C2B000E7D2301017E076E
:103E30007E29D8A4F1D7D3DF0101806F8051120011
:103E4000FFFFDDD7FFFFC5CF00F01F0E001600C03B
:103E500002F0036A000EC7B4010E021203500210F2
:103E6000D8A4F1D7C584C5B4FED7A1A602D0010E4F
:103E700001D0000E1200FFFFE6D7FFFF0101AA6F7D
:103E8000C5CF00F01F0E001600C002F0036A000E3E
:103E9000C7B4010E021203500210D8A4F1D7C58096
:103EA000C5B0FED7A1B622D00101AA5125D800097C
:103EB000D8A41CD0C5CF00F01F0E001600C002F021
:103EC000036A000EC7B4010E021203500210D8A4F8
:103ED000F1D7A1B60BD0C5BC02D0D96A02D0040E6E
:103EE000D96EC584C5B4FED7A1A602D0010E01D0FB
:103EF000D9501200FFFFC2D7FFFFC96EC6AE02D075
:103F0000FF0E03D0C7B0FED7000E1200FFFFF5D79B
:103F1000FFFFC586C7A0FED7C9501200FFFFF9D723
:103F20007601FFFF76C102F077C103F078C1F3FF9D
:103F300079C1F4FF01017A51006E7B51016E7A075D
:103F4000000E7B5B01500010D8B43CD0F3CFF6FFDD
:103F5000F4CFF7FFF32A000EF422050EF76404D025
:103F60000800FFFFF55005D0F6CFE9FFF7CFEAFFD5
:103F7000EF50016E02C0F6FF03C0F7FF022A000EE9
:103F80000322050EF76404D00800FFFFF55005D0AA
:103F9000F6CFE9FFF7CFEAFFEF50006E0150005C6B
:103FA00001017C6F7D6BD8A07D0700BE7D0701BE3F
:103FB0007D2B7D517C11D8B4BDD77CC100F07DC173
:103FC00001F002D0006A016A1200FFFFABD7FFFFC9
:103FD000D96E390ED96401D006D0300ED96001D027
:103FE00002D0D88001D0D8901200FFFFF1D7EECFD9
:103FF000E6FFE82EFCD7000CFFFF1200FFFFFDD705
:10400000FFFFE8D1CED10101066907690869096996
:104010000A690B690C690D690E690F690201456B2C
:10402000466B476B486B440E0101106F116B060E17
:10403000126F010E136F430E146F156B6AEC00F0D4
:10404000E8CFE0F5FBEC38F000C037F201C038F201
:10405000010EE8CF6FF5FBEC38F037C202F038C242
:1040600003F00350015C02E10250005CD8A02DD0A7
:1040700000D0FBEC38F037C2E8FF005C026E38C2BB
:10408000E8FF0158036E000E035C020ED8B4025C18
:10409000000ED8B0010E006E016A18D0FBEC38F0AB
:1040A00000C002F001C003F037C2F6FF38C2F7FFCC
:1040B000FF0E006EFF0E016EF650005EF750015AC3
:1040C000025000260350012201D0E8D70150001011
:1040D000D8B401D001D003D0020EE8CF6FF578D16B
:1040E00002014551461147114811D8B401D001D001
:1040F00004D0040EE8CF6FF50BD0010E38DBFBECDB
:1041000038F000C037F201C038F2030EE8CF6FF587
:104110005FD1E0C5E8FFB4EC01F00009D8B401D0EC
:1041200001D00AD064D9020AD8A401D001D003D0AA
:10413000040EE8CF6FF544D0FBEC38F037C202F044
:1041400038C203F00350015C02E10250005CD8A0C9
:104150002DD000D0FBEC38F037C2E8FF005C026ED7
:1041600038C2E8FF0158036E000E035C0A0ED8B493
:10417000025C000ED8B0010E006E016A18D0FBEC94
:1041800038F000C002F001C003F037C2F6FF38C2B9
:10419000F7FFFF0E006EFF0E016EF650005EF75047
:1041A000015A025000260350012201D0E8D70150E5
:1041B0000010D8B401D001D003D0020EE8CF6FF5C3
:1041C00007D1E0C5E1F5EFEC28F00009D8B401D043
:1041D00001D00BD0030ECBDAFBEC38F000C037F285
:1041E00001C038F2050EE8CF6FF5F2D0E0C5E8FF68
:1041F000B4EC01F00009D8B401D001D032D0F7D826
:10420000050AD8A401D001D02BD0E0C5E8FFCCEC42
:1042100000F0FBEC38F000C037F201C038F2060EB7
:10422000E8CF6FF545C21EF246C21FF247C220F228
:1042300048C221F249C228F24AC229F24BC22AF2EC
:104240004CC22BF241C22CF242C22DF243C22EF2DA
:1042500044C22FF2050170810501010EDF27B8D09D
:1042600044D0FBEC38F037C202F038C203F0035000
:10427000015C02E10250005CD8A02DD000D0FBEC24
:1042800038F037C2E8FF005C026E38C2E8FF015820
:10429000036E000E035C0A0ED8B4025C000ED8B0A8
:1042A000010E006E016A18D0FBEC38F000C002F07D
:1042B00001C003F037C2F6FF38C2F7FFFF0E006EF1
:1042C000FF0E016EF650005EF750015A02500026B4
:1042D0000350012201D0E8D701500010D8B401D01A
:1042E00001D003D0020EE8CF6FF572D0FBEC38F0AE
:1042F00037C202F038C203F00350015C02E1025001
:10430000005CD8A02DD000D0FBEC38F037C2E8FF1D
:10431000005C026E38C2E8FF0158036E000E035CB9
:104320000A0ED8B4025C000ED8B0010E006E016A0D
:1043300018D0FBEC38F000C002F001C003F037C227
:10434000F6FF38C2F7FFFF0E006EFF0E016EF6504B
:10435000005EF750015A025000260350012201D09E
:10436000E8D701500010D8B401D001D019D0020113
:10437000FF0E3927FF0E3A23FF0E3B23FF0E3C238F
:1043800039513A113B113C11D8A401D001D002D0CF
:1043900005016F6BFBEC38F000C037F201C038F25A
:1043A00017D06FC5E8FF000A01E12DD6010A01E12F
:1043B00052D6030A01E194D6010A01E1AAD6070AFE
:1043C00001E1FFD6010A01E111D7030A8FE000D015
:1043D0001200FFFF17D6FFFF09D0080EE8CF6FF5D8
:1043E000E0C5E8FFCCEC00F01200FFFFF6D7FFFFBE
:1043F000BDD10101126B0201000E3C6F000E3B6F3C
:10440000000E3A6F3C0E396F0101100E186F010E4D
:10441000196FC6EC01F001011051020AD8A401D0B5
:1044200001D078D1116B0E0E116501D001D001D0F1
:104430000FD00101100E186F010E196FC6EC01F0BC
:10444000010E010111270E0E116501D001D0F1D727
:104450000101450E186F020E196FC6EC01F0010143
:10446000460E186F020E196FC6EC01F00101470EDF
:10447000186F020E196FC6EC01F00101480E186F9B
:10448000020E196FC6EC01F00101116BDB0E116514
:1044900001D001D001D00FD00101100E186F010E14
:1044A000196FC6EC01F0010E01011127DB0E116539
:1044B00001D001D0F1D70101136B0101100E186F6B
:1044C000010E196FC6EC01F00CD10101100E186F2E
:1044D000010E196FC6EC01F001011005D8A401D03E
:1044E00001D007D0120E186F010E196FC6EC01F043
:1044F00001D038D109D10101100E186F010E196FCA
:10450000C6EC01F001011051040AD8A401D001D079
:104510001CD0490E186F020E196FC6EC01F0010194
:104520004A0E186F020E196FC6EC01F001014B0E16
:10453000186F020E196FC6EC01F001014C0E186FD6
:10454000020E196FC6EC01F001D00CD1DDD00101D3
:10455000100E186F010E196FC6EC01F0030E010169
:10456000106501D001D01CD0410E186F020E196FDA
:10457000C6EC01F00101420E186F020E196FC6EC75
:1045800001F00101430E186F020E196FC6EC01F025
:104590000101440E186F020E196FC6EC01F001D034
:1045A000E1D0FC0E0101102707D00101110E186F98
:1045B000010E196FC6EC01F0010110071029D8A4F3
:1045C00001D001D0F2D7A0D00101100E186F010E5A
:1045D000196FC6EC01F001011051040AD8A401D0F2
:1045E00001D01CD0170E186F010E196FC6EC01F028
:1045F0000101160E186F010E196FC6EC01F00101D2
:10460000150E186F010E196FC6EC01F00101140EA2
:10461000186F010E196FC6EC01F001D0A3D074D051
:10462000010E0101136F70D00101100E186F010E01
:10463000196FC6EC01F001011051040AD8A401D091
:1046400001D036D03C0E186F020E196FC6EC01F087
:1046500001013B0E186F020E196FC6EC01F001014B
:104660003A0E186F020E196FC6EC01F00101390EF7
:10467000186F020E196FC6EC01F002EE3CF0000E4E
:10468000ED5C08E1000EED5C05E1070EED5C02E17A
:10469000090EEF5CD8A001D001D009D00201F80EBC
:1046A0003927F80E3A23FF0E3B23FF0E3C2301D09F
:1046B00059D02AD00101100E186F010E196FC6ECE7
:1046C00001F007D00101110E186F010E196FC6EC31
:1046D00001F0010110071029D8A401D001D0F2D7B0
:1046E00013D001011051010A01E105D7020A01E1CD
:1046F0002ED7300A99E0060A01E1E7D6030A01E164
:1047000063D7C90A8DE0D6D701011351D8B401D0BF
:1047100001D0D3D601011251020AD8A401D001D090
:1047200009D014C13DF215C13EF216C13FF217C1C6
:1047300040F213D002EE3DF00101EE50141908E1F1
:10474000EE50151905E1EE50161902E1EE50171959
:10475000D8B401D001D001D0126BEFEC01F001010F
:10476000125102D0000E00D01200FFFF42D6FFFF10
:10477000D7D00101116F010EDBEC00F0010EDBEC74
:1047800000F0060EDBEC00F0000EDBEC00F0120E89
:10479000DBEC00F0230EDBEC00F0340EDBEC00F081
:1047A000560EDBEC00F0000EDBEC00F0000EDBEC54
:1047B00000F0800EDBEC00F0000EDBEC00F00101FD
:1047C0001151030AD8A401D001D011D045C2E8FF8D
:1047D000DBEC00F046C2E8FFDBEC00F047C2E8FF8C
:1047E000DBEC00F048C2E8FFDBEC00F00CD0000E80
:1047F000DBEC00F0000EDBEC00F0000EDBEC00F078
:10480000000EDBEC00F00101106B0B0E106501D007
:1048100001D001D00BD0000EDBEC00F0010E010145
:1048200010270B0E106501D001D0F5D722C2E8FF8A
:10483000DBEC00F023C2E8FFDBEC00F024C2E8FF71
:10484000DBEC00F025C2E8FFDBEC00F026C2E8FF5D
:10485000DBEC00F027C2E8FFDBEC00F00101106B9D
:10486000C90E106501D001D001D00BD0000EDBECD9
:1048700000F0010E01011027C90E106501D001D012
:10488000F5D7630EDBEC00F0820EDBEC00F0530E8C
:10489000DBEC00F0630EDBEC00F0350EDBEC00F03F
:1048A000010EDBEC00F001011151DBEC00F0010125
:1048B0001105D8B40AD000D0020145514611471164
:1048C0004811D8B402D000D002D000D016D0360E95
:1048D000DBEC00F0040EDBEC00F040C2E8FFDBECA8
:1048E00000F03FC2E8FFDBEC00F03EC2E8FFDBEC8B
:1048F00000F03DC2E8FFDBEC00F0370EDBEC00F02F
:10490000020EDBEC00F0010EDBEC00F0030EDBEC42
:1049100000F0FF0EDBEC00F02EEC01F01200FFFFC8
:1049200028D7FFFF15D0150E0101016F026BE6ECD1
:1049300005F0E8CFAFF50501B26B0501B06B0501DD
:10494000AD6B0201140E4D6F000E4E6F1200FFFF93
:10495000EAD7FFFF53D1AFC5E8FF13EC07F000091A
:10496000D8A401D001D00DD00501B06B070EE8CF5F
:10497000ABF50501B26B0501AD6B0501B36B010E23
:104980003BD1AFC5E8FFF4EC09F00009D8B401D081
:1049900001D04ED0FBEC38F000C051F201C052F211
:1049A00015D0B0C5E8FF05EEBEF0E926000EEA22FC
:1049B00000C1EFFF0501010EB027B0C5E8FF1F0AD7
:1049C000D8A401D001D002D00501B06B0101000EC6
:1049D000666F010E676FAFC5E8FF96EC09F0006ED9
:1049E00000C002F0036A03500210D8A401D001D025
:1049F000D8D7AFC5E8FF21EC09F0010100510A0A40
:104A0000D8A401D001D013D0B0C5E8FF05EEBEF0A8
:104A1000E926000EEA22000EEF6E0501B06BA7DA60
:104A200053C205F154C206F16CDAE8CFABF54BD0B6
:104A30000501B253D8B401D001D045D0FBEC38F019
:104A400000C001F101C002F151C200F052C201F0F8
:104A500001010150025D02E10050015DD8A01BD0B0
:104A600000D051C2E8FF015D006E52C2E8FF02595A
:104A7000016E12D051C202F052C203F0FF0E006E5E
:104A8000FF0E016E0250005E0350015A01510026D4
:104A90000251012201D0EED700C001F101C002F1A4
:104AA000070E025D080ED8B4015DD8A001D001D078
:104AB0000AD001C151F202C152F2020EE8CFABF5A9
:104AC000010EE8CFB2F58BD00501AE6BFBEC38F0F0
:104AD00000C051F201C052F200D0AFC5E8FF88EC2F
:104AE00008F00009D8B401D001D0F7D7AFC5E8FF6E
:104AF00088EC08F00009D8B401D001D03AD0AEC596
:104B0000E8FF020DEA0EF324E96E000EF420EA6ECF
:104B1000EECF03F1EDCF04F107D0010100516A6F30
:104B2000AFC5E8FFA7EC08F0010103C1F6FF04C11F
:104B3000F7FF010E0327000E0423050EF76404D0CF
:104B40000800FFFFF55005D0F6CFE9FFF7CFEAFFE9
:104B5000EF50006F0051D8A401D001D0DED7AFC50F
:104B6000E8FF99EC07F00B0EE8CFAEF5010EE8CFA9
:104B7000B2F5ABC5E8FF070AD8B401D001D02DD0FB
:104B8000ABC5E8FF3CD80009D8B401D001D01AD099
:104B9000AEC5E8FF0B0AD8B401D001D004D0040E92
:104BA000E8CFB2F509D0ABC5E8FF020AD8A401D01E
:104BB00001D002D00501B26B070EE8CFABF50501BD
:104BC000B36B0BD0AEC5E8FF0B0AD8B401D001D04F
:104BD00004D0040EE8CFB2F57FD70CD00BD0B2C50D
:104BE000E8FF000A01E170D7010AC3E0050A01E10C
:104BF00073D700D0010E00D01200FFFFACD6FFFF2C
:104C000085D00101056F6FD00501AD810501AD9320
:104C1000010EE8CFAEF50101B40E066F050E076F69
:104C200001EE08F055C2EEFF56C2EDFF0A0E0A6F04
:104C30000B6B11EC38F066D0ADC500F000B001D0C0
:104C400001D004D0060EE8CFAEF520D00101B40E9D
:104C5000066F050E076F01EE08F055C2EEFF56C253
:104C6000EDFF7AEC15F0006E00C002F0036A03500D
:104C70000210D8B401D001D006D00501AD83020ED8
:104C8000E8CFAEF503D0060EE8CFAEF53BD03FD867
:104C90003BD05DC226F15EC227F1F0EC36F000C0D9
:104CA0004EF25FC226F160C227F1F0EC36F000C090
:104CB0004DF20A0EE8CFAEF525D07ED825D00A0EEB
:104CC000E8CFAEF5ACC5E8FFFE0AD8B401D001D0FC
:104CD00004D0ACC5E8FF24EC07F014D0050EE8CFF3
:104CE000AEF510D00FD001010551000A8DE0010A88
:104CF000A3E0030ACCE0010AE0E0070ACAE0010AE7
:104D0000DEE0ECD7010E00D01200FFFF7AD7FFFFE4
:104D100052D044D0B3C5E8FF020AD8A401D001D0D4
:104D200002D065EC33F0ACC5E8FFFE0AD8B401D080
:104D300001D00AD065EC33F0ACC5E8FF24EC07F0F5
:104D4000010EE8CFB3F501D00AD031D0ACC5E8FFF1
:104D500013EC07F00009D8A401D001D006D0030E4F
:104D6000E8CFAEF5030EE8CFB3F521D0AFC5E8FF2D
:104D700088EC08F00009D8B401D001D00DD0AFC53F
:104D8000E8FF13EC07F00009D8B401D001D004D03B
:104D9000AFC5E8FF24EC07F00AD009D0B3C5E8FF9F
:104DA000000AB8E0010AD2E0020AE0E000D0000EFA
:104DB00000D01200FFFFADD7FFFFA1D092D0ADC54C
:104DC00000F000B201D001D006D0060EE8CFAEF55B
:104DD000010E93D01AD0070EE8CFAEF5AFC5E8FFAD
:104DE000220D1D0EF3240101076F000EF420086F41
:104DF00001EE09F04DC2EEFF4EC2EDFF40EC06F0B1
:104E0000E8CFACF5010EE8CFB3F575D0ACC5E8FF3F
:104E100013EC07F00009D8B401D001D00FD0050180
:104E20007753D8A401D001D009D0BCEC33F000C036
:104E30004FF201C050F2020EE8CFB3F55CD0ACC522
:104E4000E8FFF4EC09F00009D8B401D001D02FD06C
:104E5000FBEC38F000C051F201C052F24FC2A9F190
:104E600050C2AAF1C6EC33F004D001010651E3ECC4
:104E700033F00101060E666F010E676FACC5E8FFE7
:104E800096EC09F0006E00C002F0036A03500210B5
:104E9000D8A401D001D0E9D703EC34F000C04FF220
:104EA00001C050F2ACC5E8FF21EC09F019D0ACC547
:104EB000E8FF13EC07F00009D8A401D001D010D00E
:104EC00003EC34F065EC33F0ACC5E8FF24EC07F0FC
:104ED000FE0EE8CFACF5090EE8CFAEF5010E0DD011
:104EE0000AD0B3C5E8FF000A01E169D7010A8EE0E4
:104EF000030AA5E000D0000E00D01200FFFF5ED72D
:104F00000501FFFF33D00101076B050E076501D0D6
:104F100001D001D027D005C176F106C177F101019A
:104F20000751020DDE0EF324E96E000EF420EA6E46
:104F3000EECF78F1EDCF79F1040E7A6F7B6B91ECC7
:104F40001FF001500010D8A401D001D003D00101FE
:104F500007510AD0010E01010727050E076501D090
:104F600001D0D9D7060E00D01200FFFFCCD7FFFF2B
:104F700081D00101086BBE0E056F050E066F05D0CE
:104F8000010E01010527000E062305C1E9FF06C138
:104F9000EAFFEF50200AD8B401D001D0F1D705C103
:104FA00053F206C154F2010EE8CFB1F555D048D006
:104FB00001010751200AD8A401D005D007512C0ABD
:104FC000D8A402D000D002D000D00AD005C1E9FF99
:104FD00006C1EAFF000EEF6E010E0101086F14D04A
:104FE000010107510D0AD8A401D005D007510A0AC2
:104FF000D8A402D000D002D000D006D005C1E9FF6D
:1050000006C1EAFF000EEF6E22D001010751200A0F
:10501000D8B401D001D012D0B1C5E8FF020D530EB3
:10502000F324E96E020EF420EA6E05C1EEFF06C11C
:10503000EDFF0501010EB1270101086B08D007D073
:1050400001010851000AB4E0010ADFE000D0010EBE
:1050500001010527000E062305C1E9FF06C1EAFF8D
:10506000EF500101076F0751D8A401D001D09FD79D
:105070001200FFFF7ED7FFFFD96AD950020DFE0E46
:10508000F324E96E010EF420EA6ED9CF00F0D89037
:105090000036D8900034400FEF6ED950020DFF0E4D
:1050A000F324E96E010EF420EA6E010EEF6ED92AA8
:1050B000000ED964E2D70501736BD0DA020E19EC49
:1050C00039F01F0EEDDA0101D16F1F0EDADA020E90
:1050D00019EC39F0070EE4DA006E00AE7DD0210E37
:1050E0000101D16F000ECDDA020E19EC39F0480E35
:1050F0000101D16F0E0EC5DA0101D16B0A0EC1DAC2
:105100000101D16B0B0EBDDA040E0101D16F0C0E43
:10511000B8DA020E0101D16F0D0EB3DA73C5E8FFE4
:10512000020DFE0EF324E96E010EF420EA6EEF503C
:105130000101D16F040EA5DA440E0101D16F010EF9
:10514000A0DA5F0E0101D16F020E9BDA5E0E010143
:10515000D16F030E96DA0101D169070E92DA0101CF
:10516000D16B0F0E8EDA610E0101D16F000E89DA5C
:1051700022C2D1F1010E85DA23C2D1F1020E81DA09
:1051800024C2D1F1030E7DDA25C2D1F1040E79DA01
:1051900026C2D1F1050E75DA27C2D1F1060E71DAF9
:1051A0000101006B0101D1690051080F6ADA0101A8
:1051B000002B070E0065F6D7440ED16F070E61DA9B
:1051C000440EE8CF74F5220E0101D16F000E59DABA
:1051D0000101D16B0D0E55DA1200FFFF4DD7FFFF15
:1051E000040E5EDA010B1200FFFFFAD7FFFF010188
:1051F000CB6F010ED16F0A0E44DA0101D16B0B0E99
:1052000040DA120E0101D16F000E3BDA0101CB51E1
:10521000D16F100E36D2FFFFEAD7CB01FFFF010E90
:10522000CDC100F0CEC101F00016016A0101CD51DF
:105230000024CF6FCE510120D06F400ED16F070EEA
:1052400020DA0101CF51D16F0A0E1BDA0101D051D2
:10525000D16F0B0E16DA120E0101D16F000E11DAAA
:105260000101CD51006ECE51016ECD07000ECE5B17
:1052700001500010D8B40CD0CBC1E9FFCCC1EAFF7B
:10528000EF50D16FCB2B000ECC23100EFAD9E8D7FC
:105290000101CD69CE6B04D00101CD07D8A0CE07A6
:1052A0000101CE51CD11D8B405D0070EF9D9006E49
:1052B00000ACF2D71200FFFFB2D7FFFF010E0101D1
:1052C000D16F0A0EDED90101D16B0B0EDAD90A0EAD
:1052D0000101D16F000ED5D9100EE2D1FFFFEED73C
:1052E0004001FFFF42C144F143C145F1400E0101BD
:1052F000D16F070EC6D901014451D16F0A0EC1D931
:1053000001014551D16F0B0EBCD90A0E0101D16FBD
:10531000000EB7D901014251006E4351016E4207A0
:10532000000E435B01500010D8B40CD0100EB8D959
:1053300040C1E9FF41C1EAFFEF6E0101402B000EC1
:105340004123E8D744C100F045C101F01200FFFF3E
:10535000C9D7FFFFD96E020DFF0EF324E96E010ECF
:10536000F420EA6E000EEF6A1200FFFFF3D7FFFF92
:10537000D96E020DFF0EF324E96E010EF420EA6EE1
:10538000010EEF6ED9CF73F51200FFFFF1D7FFFFCB
:105390000501740501016B6F440E6B6102D05E0E56
:1053A0006B6F200E0101D16F000E6BD901016B51A3
:1053B000D16F030E66D1FFFFEBD7FFFF600E010137
:1053C000D16F000E5ED9070E6BD90101AA6F200EB6
:1053D000D16F000E56D972C5E8FF0101AA6105D050
:1053E0005F08006EAA51002404D072C5E8FF0101D5
:1053F000AA5DD96E1B08D96E0101AC6FAB6BABC156
:1054000000F0ACC101F01200FFFFD8D70601FFFF8A
:1054100008C1E9FF09C1EAFFFF0EEF6E070E40D990
:10542000006E00A823D0210E0101D16F000E29D9F2
:10543000FF0E5BD90101D16B0A0E23D90101D16B9B
:105440000B0E1FD9020E0101D16F0D0E1AD9200EBD
:105450000101D16F000E15D99ADF0101D169070E44
:1054600010D90101D16B0D0E0CD96AD0600E01016B
:10547000D16F000E06D9070E13D901010A6F200E55
:10548000D16F000EFED801010A5105017419D8B47C
:1054900057D074C50CF101010B6B0BC1CBF10CC1E2
:1054A000CCF10DD901010D0E406F010E416F120EAE
:1054B000426F436B16DF01010DA13CD001EE0FF0EE
:1054C000EE52000EED5C400ED8B4EF5CD8A032D0A6
:1054D00001EE0FF0EE52050EED5CEF0ED8B4EF5C6E
:1054E000D8B028D01DC1C5F11EC1C6F135EC35F0CC
:1054F00000C01DF101C01EF106C146F107C147F110
:105500000101170E486F010E496F060E4A6F4B6B73
:1055100056EC38F001011E51080AD8A40BD01D51D9
:10552000D8A4060AD8A406D008C1E9FF09C1EAFF39
:105530001DC1EFFF74C572F50EC174F5010E01D0E7
:10554000000E1200FFFF64D7C301FFFF0A0E010126
:10555000D16F070E96D873C5E8FF020DFE0EF32437
:10556000E96E010EF420EA6EEF500101CA6FC96BBB
:10557000C9C1CBF1CAC1CCF1A2D8C3C1CBF1C4C15E
:10558000CCF1060E0101CD6FCE6B48DE22C2E8FFE2
:105590002DDE23C2E8FF2ADE24C2E8FF27DE25C273
:1055A000E8FF24DE26C2E8FF21DE27C2E8FF1EDE78
:1055B0000101C551D8A402D0C86B03D0060E010169
:1055C000C86F080E13DE0101C85110DE0E0E010176
:1055D000C627000EC723C75D3C0ED8B4C65DD8B041
:1055E00003D0400EC66FC76BC6C1C9F1C7C1CAF1AF
:1055F0000101C951D16F050E44D80101CA51D16FC3
:10560000060E3FD0FFFFA2D7FFFF73C5E8FF020DD4
:10561000FE0EF324E96E010EF420EA6EEF50010154
:10562000D16F040E2ED8240E0101D16F000E29D89F
:10563000D96AD950020DFF0EF324E96E010EF42051
:10564000EA6EEF50D8B403D0D9CF73F504D0D92A7D
:10565000000ED964EED71200FFFFD7D7FFFF956881
:10566000816AE00E936EF19E848284808484966ABF
:10567000010ED96ED92EFED784941200FFFFEFD70A
:10568000D101FFFFD96E816EE00E936E0101D15101
:10569000836E956A8492848295681200FFFFF2D728
:1056A000FFFFE16E9568E150816EE00E936E84908D
:1056B0008350D96E84801200FFFFF3D7CB01FFFF28
:1056C000CBC1CDF1CCC1CEF1400E0101D16F070E9F
:1056D000D8DF0101CD51D16F080ED3DF0101CE51CA
:1056E000D16F090ECED7FFFFEBD7FFFF0101206F6F
:1056F0001F6B01011F51006E2051016E1F07000E2C
:10570000205B01500010D8B41200F3D7FFFFEED792
:105710006A01FFFF72C56DF1120E01016C6F6A51D3
:105720006C276B516D236CC1CBF16DC1CCF1C7D728
:10573000FFFFF0D7AA01FFFFE16EE1CF73F573C55C
:10574000E8FF020DFE0EF324E96E010EF420EA6E6E
:10575000EF500101AD6F0E0EAC6FAA51AC27AB51EB
:10576000AD23ACC1CBF1ADC1CCF1A9D7FFFFE4D7DC
:105770002B01FFFF0101396B3A6B2BC137F12CC1B3
:1057800038F101012FC1F6FF30C1F7FF2F2B000EBA
:105790003023050EF76404D00800FFFFF55005D054
:1057A000F6CFE9FFF7CFEAFFEF50346F3451010134
:1057B000D8B4C8D2250AD8B40BD0392B000E3A235E
:1057C0002E512D11D8A47BD13451FCEC1FF0D9D728
:1057D00001013269336B316B63D201012E512D11FE
:1057E000D8A4B4D2B9D237C1E9FF38C1EAFF010168
:1057F000020E3727000E3823EF5096D20101318D6B
:105800004FD20101312B06D0080E01013227FE0EC6
:105810000101322737C1E9FF38C1EAFF0101020E59
:105820003727000E3823EECF35F1EDCF36F131A119
:105830000DD036AF06D0356D361FD8B0362B3307B6
:1058400007D00101319131AD03D0F9D70101319178
:105850000B0E0101322732C102F0036A35C100F09C
:1058600036C101F08CEC38F000500101346F32C1C8
:1058700002F0036A35C100F036C101F08CEC38F05B
:1058800004C035F105C036F1010E3B6F3C6B0101E0
:105890003C51365D02E13B51355DD8A010D032C19C
:1058A00002F0036A3BC100F03CC101F04DEC39F05D
:1058B00004C03BF105C03CF101013307E8D7010109
:1058C00031A916D01CD00101392B000E3A232E51DC
:1058D0002D11D8B40AD02DC1E9FF2EC1EAFF200E48
:1058E000EF6E2D2B000E2E2303D0200EFCEC1FF0AC
:1058F000010133073351800A7F0FD8B0E4D701018B
:1059000031A115D0392B000E3A232E512D11D8B4C8
:105910000AD02DC1E9FF2EC1EAFF2D0EEF6E2D2B0F
:10592000000E2E2317D02D0EFCEC1FF013D001011A
:1059300031AD10D0392B000E3A232E512D11D8B491
:1059400006D02DC1E9FF2EC1EAFF2B0EE7D72B0EA3
:10595000FCEC1FF0010131B916D051D00101392BF7
:10596000000E3A232E512D11D8B40AD02DC1E9FFD3
:105970002EC1EAFF300EEF6E2D2B000E2E2303D02A
:10598000300EFCEC1FF0010133073351800A7F0F0A
:10599000D8A035D0E3D73BC102F03CC103F035C1FC
:1059A00000F036C101F08CEC38F004C000F005C006
:1059B00001F032C102F0036A8CEC38F000500101B2
:1059C000336F800A760FD8A002D0070E332701016B
:1059D000392B000E3A232E512D11D8B40BD0335150
:1059E000300F2DC1E9FF2EC1EAFFEF6E2D2B000E07
:1059F0002E2305D001013351300FFCEC1FF032C1D2
:105A000002F0036A3B0EE96E010EEA6EEE50006E84
:105A1000EF50016E8CEC38F00550ED6E0450EF6ED7
:105A2000EE50ED10D8A4B7D7090E0101346502D0AD
:105A3000070E34270101392B000E3A232E512D1168
:105A4000D8B408D03451300F2DC1E9FF2EC1EAFF80
:105A5000EF6E3BD001013451300FFCEC1FF091D6BA
:105A600001013351800A7E0FD8A017D0392B000EC8
:105A70003A232E512D11D8B40AD02DC1E9FF2EC1E1
:105A8000EAFF200EEF6E2D2B000E2E2303D0200EEA
:105A9000FCEC1FF001013307E3D737C1E9FF38C140
:105AA000EAFF0101020E3727000E3823EF50346F52
:105AB000392B000E3A232E512D11D8B40AD02DC106
:105AC000E9FF2EC1EAFF34C1EFFF2D2B000E2E237C
:105AD00058D601013451FCEC1FF053D637C1E9FF11
:105AE00038C1EAFF0101020E3727000E3823EECF3E
:105AF00000F0EDCF01F000C0FAF101C0FBF1D96A6E
:105B0000D9CF00F0016AFAC1E8FF0024026EFBC1A0
:105B1000E8FF0120036E02C0F6FF03C0F7FF050E89
:105B2000F76404D00800FFFFF55005D0F6CFE9FF79
:105B3000F7CFEAFFEF500009D8B402D0D92AE0D756
:105B400001013251D96002D0D950326F0101325176
:105B500033BF46D0FF0A3325D8A042D0392B000EE0
:105B60003A232E512D11D8B40AD02DC1E9FF2EC1F0
:105B7000EAFF200EEF6E2D2B000E2E2303D0200EF9
:105B8000FCEC1FF001013307E1D7FAC1F6FFFBC1BE
:105B9000F7FF050EF76404D00800FFFFF55005D0AD
:105BA000F6CFE9FFF7CFEAFFEF500101346F0101B3
:105BB000FA2B000EFB230101392B3A232E512D1114
:105BC000D8B40AD02DC1E9FF2EC1EAFF34C1EFFFDE
:105BD0002D2B000E2E2304D001013451FCEC1FF0BC
:105BE000010132073229D8B4CCD5CFD72FC1F6FF67
:105BF00030C1F7FF050EF76404D00800FFFFF55031
:105C000005D0F6CFE9FFF7CFEAFFEF502A0AD8A474
:105C10000FD037C1E9FF38C1EAFF0101020E372773
:105C2000000E3823EF50326F2F2B000E302338D068
:105C30002FC1F6FF30C1F7FF050EF76404D008004E
:105C4000FFFFF55005D0F6CFE9FFF7CFEAFFEF50A1
:105C5000D00F0101326F2F2B000E30232FC1F6FF22
:105C600030C1F7FF050EF76404D00800FFFFF550C0
:105C700005D0F6CFE9FFF7CFEAFFEF50D96E2F0E30
:105C8000D9640ED03A0ED9600BD0010132510A0D01
:105C9000D950F324D00FC7D7010131B538D031899D
:105CA00001012FC1F6FF30C1F7FF2F2B000E30236B
:105CB000050EF76404D00800FFFFF55005D0F6CFBD
:105CC000E9FFF7CFEAFFEF50346F000A01E185D515
:105CD0002A0A01E188D5010A01E190D5050A86E08A
:105CE0001E0ADAE0680A01E18FD53B0A01E1B8D665
:105CF000070A01E186D50B0A01E189D51C0A01E1F9
:105D0000EDD6060A01E186D50D0A01E17DD52F0EFB
:105D1000010134650BD03A0E346108D0318533511E
:105D20000A0D3451F324D00F336FBAD70101392B48
:105D3000000E3A232E512D11D8A4C1D63451FCECBB
:105D40001FF01FD52E512D11D8B406D02DC1E9FF5B
:105D50002EC1EAFF000EEF6A39C100F03AC101F02E
:105D60001200FFFF07D50601FFFF01012B0E406F58
:105D7000010E416F140E426F436B71EC29F001016B
:105D80002B51F00B400AD8A4B0D02BC100F00F0E5D
:105D90000016D8900036D8900034EC0F0E6F140E19
:105DA0000E6501D0A2D001010E51D8B409D0170E52
:105DB000406F010E416F0E51426F436B71EC29F041
:105DC00035C111F136C112F10101356B366B2B0E65
:105DD000C36F010EC46F140EC56FC66B92EC35F025
:105DE000001C026E011C036E02C013F103C014F10B
:105DF00001010E51D8B412D0170EC36F010EC46F3B
:105E00000E51C56FC66B92EC35F0001C026E011C82
:105E1000036E02C015F103C016F103D00101156B2A
:105E2000166B0101130EC36F010EC46F040EC56F14
:105E3000C66B92EC35F000C00FF101C010F101010A
:105E40002B0EC36F010EC46FBCD801011051121983
:105E500002E10F511119D8A448D02B51F00B400A80
:105E6000D8A443D006C1E1FF07C1E2FFE250E11030
:105E7000D8B40CD0E1CFE9FFE2CFEAFF3BC1EEFF9F
:105E80003CC1EEFF3DC1EEFF3EC1EEFF010100EE61
:105E900006F00851E9260951EA2237C1EEFF38C160
:105EA000EEFF39C1EEFF3AC1EEFF0AC1E9FF0BC1B7
:105EB000EAFF34C1EFFF0E5101EE2DF0EECF00F0FE
:105EC000EDCF01F0005E000E015AEC0E0024006ED2
:105ED000FF0E0120016E0CC1E9FF0DC1EAFF00C0F9
:105EE000EEFF01C0EDFF010E03D0C7EC29F0000E5C
:105EF0001200FFFF3AD7AA01FFFF450E0101AF6F65
:105F0000B06B140EAD25B16F000EAE21B26F010162
:105F1000F82B000EF92301EEB3F0F8C1EEFFF9C142
:105F2000EDFF0101B56BB66B640EB76FAC51B86F86
:105F3000B96BBA6B1EC2BBF11FC2BCF120C2BDF16E
:105F400021C2BEF100EE06F0AA51E926AB51EA22C9
:105F5000EECFBFF1EECFC0F1EECFC1F1EECFC2F187
:105F6000AF0EC36F010EC46F2CD80101AF0EC36F0B
:105F7000010EC46F140EC56FC66B92EC35F000C0F5
:105F8000B9F101C0BAF1AAC1C3F1ABC1C4F10101B9
:105F9000C56B140EAD25C66F000EAE21C76FA5EC04
:105FA0002AF00101AF0ECB6F010ECC6F140ECD6F36
:105FB000CE6B0EEC29F0006A016A1200FFFF9DD73C
:105FC000C301FFFF010100EE02F0C351E926C451F5
:105FD000EA22EECFC5F1EDCFC6F135EC35F0010187
:105FE00000EE02F0C351E926C451EA2200C0EEFFE0
:105FF00001C0EDFF00EE04F0C351E926C451EA22CE
:10600000EECFC5F1EDCFC6F135EC35F0010100EE74
:1060100004F0C351E926C451EA2200C0EEFF01C0DA
:10602000EDFF00EE0AF0C351E926C451EA22EECF9B
:10603000C5F1EDCFC6F135EC35F0010100EE0AF007
:10604000C351E926C451EA2200C0EEFF01C0EDFFB2
:106050001200FFFFB7D71101FFFF0101150E406FBE
:10606000010E416F1C0E426F436B71EC29F0C7ECBF
:1060700029F00101150E316F010E326F10D901EEBA
:1060800015F0EE50010AED10D8A453D001011951BA
:10609000060AD8A44ED01A51040AD8A44AD013C173
:1060A000E1FF14C1E2FF11C1D9FF12C1DAFF01EE15
:1060B0001BF0EE50020AED10D8A402D0000E08D05A
:1060C00001EE1BF0EE50010AED10D8A403D0010E32
:1060D000E76E03D0020EE76E2CD01EC2E8FF01016E
:1060E0002D6327D01FC2E8FF2E6323D020C2E8FF14
:1060F0002F631FD021C2E8FF30631BD01D0EE96E55
:10610000010EEA6ED9CFE1FFDACFE2FF060EF7EC1F
:106110001FF000EE06F0D950E926DA50EA2223C13A
:10612000EEFF24C1EEFF25C1EEFF26C1EEFF010EFA
:1061300001D0000E1200FFFF90D71101FFFF11C127
:10614000D9FF12C1DAFF010E0101146F156B166B36
:10615000080E176F060E186F040E196F1305D8A4DA
:106160000AD0010E1A6F1B6B2669276928692969F5
:106170002A692B690FD0020E01011A6F1B6BD9CF50
:10618000E9FFDACFEAFF260EE16E010EE26E060E9F
:10619000F7EC1FF022C21CF123C21DF124C21EF134
:1061A00025C21FF126C220F127C221F11EC222F111
:1061B0001FC223F120C224F121C225F128C200F020
:1061C00000EE06F0D950E926DA50EA22EF5001013C
:1061D0002219016E0014D8A42AD029C200F000EEC2
:1061E00007F0D950E926DA50EA22EF502319016E60
:1061F0000014D8A41CD02AC200F000EE08F0D95038
:10620000E926DA50EA22EF502419016E0014D8A4CE
:106210000ED02BC200F000EE09F0D950E926DA507A
:10622000EA22EF502519016E0014D8B409D02CC20F
:106230002CF12DC22DF12EC22EF12FC22FF10ED036
:1062400000EE06F0D950E926DA50EA22EECF2CF122
:10625000EECF2DF1EECF2EF1EECF2FF10101140E86
:10626000316F010E326F1BD80101260EC36F010E74
:10627000C46F060EC56F1C0EC66FC76BA5EC2AF067
:106280000101140ECB6F010ECC6F1C0ECD6FCE6BC7
:106290000EEC29F004EF2BF0FFFF51D73101FFFF87
:1062A00031C1E9FF32C1EAFFEECFC5F1EDCFC6F152
:1062B00035EC35F031C1E9FF32C1EAFF00C0EEFF35
:1062C00001C0EDFF010100EE02F03151E92632512B
:1062D000EA22EECFC5F1EDCFC6F135EC35F0010184
:1062E00000EE02F03151E9263251EA2200C0EEFF01
:1062F00001C0EDFF00EE06F03151E9263251EA22ED
:10630000EECFC5F1EDCFC6F135EC35F0010100EE71
:1063100006F03151E9263251EA2200C0EEFF01C0F9
:10632000EDFF1200FFFFBCD7FFFF0501786B0501F1
:1063300079813BEC28F041EC36F056EC00F08EEF22
:1063400005F0FFFFF2D7FFFF010E0101006F010111
:106350000051D8B429D1006B0ED10101670E066F30
:10636000020E076F010E086F010E096F07EC2AF08D
:10637000006E00C002F0036A03500210D8B4E7D7E1
:10638000010E0101006F0151D8A402D0020E5DD0B0
:1063900001010151060AD8A402D0050E56D0C7EC5F
:1063A00029F0D5D70101006B54EC36F00009D8B4C0
:1063B000CED752D00101020E066F010E076F670E95
:1063C000086F020E096F010E0A6F010E0B6F610E4E
:1063D0000C6F020E0D6FB4EC2EF0006E00C002F0D8
:1063E000036A03500210D8B43AD0010E0101006FC5
:1063F0000105D8A41DD0030EE8CF78F579C500F0CB
:1064000000A0A5D70229D8B40329D8B40429D8B448
:106410000529D8B49CD70501799102C11EF203C1A8
:106420001FF204C120F205C121F2EBEC21F08FD75D
:1064300001010151060AD8A402D0060E06D00101BE
:106440000151110AD8A404D0070EE8CF78F57FD700
:106450000101006BC7EC29F00501786B78D7C7EC18
:1064600029F0FAD70101670E066F020E076F01EEE1
:1064700008F061C2EEFF62C2EDFF0EEC02F0006EAA
:1064800000C002F0036A03500210D8B402D0050124
:10649000786B0101006B5BD70101670E066F020E7E
:1064A000076F01EE08F061C2EEFF62C2EDFF0AEC79
:1064B0000AF0006E00C002F0036A03500210D8A474
:1064C000E6D7E7D70501786B0201000E625D2A0E60
:1064D000D8B4615DD8B02CD00101010E066F010E59
:1064E000076F7A0E086F050E096F610E0A6F020EB4
:1064F0000B6F630E0C6F020E0D6F650E0E6F020EAA
:106500000F6F16EC34F0006E00C002F0036A035007
:106510000210D8B40BD001010151080AD8A406D04A
:10652000010E006F040EE8CF78F502D00501786BFC
:10653000C7EC29F00CD7EFEC28F000090101D8B422
:1065400007D7670E066F020E076F086B7A0E096F8A
:10655000050E0A6F61C20BF101EE0CF063C2EEFF93
:1065600064C2EDFF01EE0EF065C2EEFF66C2EDFF04
:1065700096EC34F071D778C5E8FF000A01E1EDD65A
:10658000010A01E1EAD6030A01E114D7010A9AE0FF
:10659000070AD1E0010A01E105D7030A01E17CD72E
:1065A000010A01E15FD7D3D605EC0AF000EC20F038
:1065B00070C500F000A002D0050179911200FFFF24
:1065C000C3D6FFFF0501776B0501766B0B0EDCEC84
:1065D0001DF0010CFFFFF6D76601FFFF76C500F046
:1065E00000A003D0006A016A6DD0200E0101696F1E
:1065F0006A6B66C1E9FF67C1EAFFEF50D8B45FD0AC
:1066000066C17AF167C17BF1F6EC35F000C066F146
:1066100001C067F169C17AF16AC17BF101016B0EBA
:106620007C6F010E7D6F0F0E7E6FA00EFEEC1EF0D4
:1066300001016B51D8A42FD066C17AF167C17BF1FB
:10664000C0EC38F000500101686F0C0E686501D095
:10665000686F66C17AF167C17BF101016E0E7C6FD4
:10666000010E7D6F68517E6F7F6B9AEC37F00150A1
:106670000010D8A40AD00501010E772B01EE6CF0B2
:10668000EECF00F0EDCF01F01DD00F0E0101692714
:10669000000E6A23BFD701016B51040AD8A40FD0A2
:1066A00001EE6CF0EE52ED50FF0AFF0ED8B4EF1879
:1066B000D8B405D06CC169F16DC16AF1ABD7FF0EDA
:1066C000006801681200FFFF89D7FFFF0501756BA5
:1066D0000501769105017753D8B402D0010E7707F2
:1066E0001200FFFFF3D76A01FFFF6AC1FCF16BC123
:1066F000FDF16AC181F16BC182F1A00E54EC1EF074
:10670000006E00C002F0036A03500210000ED8B4FD
:10671000010E1200FFFFE9D7FFFFE3EC1EF00101BD
:106720006A6F0101FC2B000EFD2301016A51030A6F
:10673000D8A409D0E3EC1EF001016A6F0101FC2B23
:10674000000EFD230AD001016A51040AD8A405D025
:10675000FF0EE8CFFCF1E8CFFDF101016A51120014
:10676000FFFFDBD7FFFFEFEC1EF0FCC100F0FDC127
:1067700001F01200FFFFF7D7FFFF05017681200E21
:10678000006E016A1200FFFFF8D7A901FFFFA9C13F
:10679000FCF1AAC1FDF1A9C175F505013F0E751700
:1067A000A9C1ABF1AAC1ACF1A00EEDEC1DF0006ED9
:1067B00000C002F0036A03500210000ED8B4010EAC
:1067C0001200FFFFE4D7FFFF0101A96F9CEC1EF050
:1067D0000009D8B402D0000E13D00501752B0101B9
:1067E000FC2B000EFD233F0E0501756508D00BD86C
:1067F000FCC1ABF1FDC1ACF1A00EEDEC1DF0010E42
:106800001200FFFFE1D7FFFF0501756BCDEC1EF015
:10681000A00E3DEC1FF00009D8A4FAD7FCC100F08F
:10682000FDC101F01200FFFFEFD70601FFFF0101DC
:10683000180E406F010E416F080E426F436B71ECF2
:1068400029F01AC112F11BC113F101011A6B1B6B64
:10685000180EC36F010EC46F080EC56FC66B92ECA5
:1068600035F0001C026E011C036E02C014F103C05F
:1068700015F10AC1E1FF0BC1E2FFF80EE72608C1DE
:1068800040F109C141F1E7500101426F436B71ECE6
:1068900029F008C1C3F109C1C4F10AC1E9FF0BC164
:1068A000EAFFEF500101C56FC66B92EC35F0001C9A
:1068B000026E011C036E02C016F103C017F1010144
:1068C000140EC36F010EC46F040EC56FC66B92EC3D
:1068D00035F000C010F101C011F10101180E406F38
:1068E000010E416F77D806C1E9FF07C1EAFF18C161
:1068F000EFFF0CC1E9FF0DC1EAFF1CC1EEFF1DC196
:10690000EDFF0EC1E9FF0FC1EAFF1EC1EEFF1FC17F
:10691000EDFF01011351111902E112511019000E7E
:10692000D8B4010E1200FFFF82D70601FFFF01015C
:10693000116B0851106F126B136B0CC114F10DC168
:1069400015F10EC116F10FC117F1180E466F010EA9
:10695000476F09C148F10AC149F10B514A6F4B6BAE
:1069600056EC38F00101100E406F010E416F32D825
:106970000101100EC36F010EC46F080E0B25C56F09
:10698000C66B000EC62392EC35F000C012F101C0B8
:1069900013F106C1AAF107C1ABF1010E0101AC6F01
:1069A000080E0B25AD6FAE6B000EAE237CEC2FF006
:1069B0000101100ECB6F010ECC6F080E0B25CD6FB1
:1069C000CE6B000ECE230EEC29F004EF2BF0FFFF70
:1069D000AED74001FFFF010100EE04F04051E9266F
:1069E0004151EA22EECFC5F1EDCFC6F135EC35F0DD
:1069F000010100EE04F04051E9264151EA2200C0B5
:106A0000EEFF01C0EDFF00EE06F04051E9264151D6
:106A1000EA22EECFC5F1EDCFC6F135EC35F001013C
:106A200000EE06F04051E9264151EA2200C0EEFF97
:106A300001C0EDFF00EE02F04051E9264151EA228B
:106A4000EECFC5F1EDCFC6F135EC35F0010100EE2A
:106A500002F04051E9264151EA2200C0EEFF01C098
:106A6000EDFF1200FFFFB7D7C501FFFFC5C1C7F19A
:106A7000C6C1C8F10101C851D96EC751C86FD950FC
:106A8000C76FC7C100F0C8C101F01200FFFFEED709
:106A9000AC01FFFFACC1B0F1ADC1B1F1AEC1B2F11B
:106AA000AFC1B3F1B00ED96E010EDA6E00EE03F095
:106AB000D950E926DA50EA22EF50F36E00EE03F0E7
:106AC000D950E926DA50EA22DFCFEFFFF3CFDFFF1C
:106AD00000EE02F0D950E926DA50EA22EF50F36EC8
:106AE00010EE01F0D950E126DA50E22200EE02F079
:106AF000D950E926DA50EA22E7CFEFFF00EE01F0A5
:106B0000D950E926DA50EA22F3CFEFFFB0C100F006
:106B1000B1C101F0B2C102F0B3C103F01200FFFF36
:106B2000B9D7C301FFFF0101CB6BCC6BCD6BCE6B33
:106B3000D890C631F46EC531F36EC3C1E1FFC4C154
:106B4000E2FFF350006EF450016EF306000EF45AAB
:106B500001500010D8B418D0E1CFE9FFE2CFEAFF2E
:106B6000020EE126000EE222EECF00F0EDCF01F0A2
:106B7000026A036A01010050CB270150CC23025066
:106B8000CD230350CE23DDD70101C5A109D0E750A5
:106B9000CB27010ED8B0CC27D8B0CD27D8B0CE2780
:106BA000CBC1C7F1CCC1C8F1CDC1C9F1CEC1CAF1C9
:106BB000C9C1F3FFCAC1F4FFF450F3100101D8B406
:106BC0000DD0CD6BCE6BCB51F324CB6FCC51F420D9
:106BD000CC6FCD6BD8B0CD2BCE6BE2D7CB1D006E7A
:106BE000CC1D016E1200FFFF9ED77A01FFFF7AC114
:106BF000E1FF7BC1E2FFE750D96ED950D8B40AD08B
:106C0000600ED96405D07B0ED96002D0E00EE72675
:106C1000E652F1D77AC100F07BC101F01200FFFF0C
:106C2000E6D77601FFFF78C1F3FF79C1F4FF76C1A3
:106C3000D9FF77C1DAFF01017A077A29D8B41AD0CF
:106C4000F3CFF6FFF4CFF7FFF32A000EF422D9CFEB
:106C5000E9FFDACFEAFFD94ADA2A050EF76403D052
:106C60000800F55005D0F6CFE1FFF7CFE2FFE7507F
:106C7000EF6EE1D776C100F077C101F01200FFFF9F
:106C8000D2D7FFFF0501716BFF0EE8CF71F2E8CF9D
:106C900072F2E8CF73F2E8CF74F2E8CF75F2E8CF82
:106CA00076F21200FFFFEED7FFFF32D00101070E90
:106CB000116F010E126F060E136F010E146F2CEC84
:106CC00030F0006E00C002F0036A03500210D8B426
:106CD00032D001010651D8A415D007C171F208C104
:106CE00072F209C173F20AC174F20BC175F20CC1E0
:106CF00076F20DC177F20EC178F20FC179F210C1B0
:106D00007AF219D0010EE8CF71F506D0000E14D03A
:106D100071C5E8FF000ACAE0EFEC28F00009D8B41A
:106D2000F5D70101070E116F010E126F136B9EEC68
:106D300030F00501716B010E1200FFFFB6D70001A4
:106D4000FFFF00C1E9FF01C1EAFFEECF06F1EECF80
:106D500007F1EECF08F1EECF09F10101000E116F3E
:106D6000010E126F010E136F9EEF30F0FFFFE9D797
:106D70000001FFFF00C1E9FF01C1EAFF02017751F5
:106D8000EE1808E17851EE1805E17951EE1802E1AC
:106D90007A51EE18D8B412D02CC2E8FF77631BD01A
:106DA0002DC2E8FF786317D02EC2E8FF0201796395
:106DB00012D02FC2E8FF02017A630DD0710EE96E86
:106DC000020EEA6E02C1E1FF03C1E2FF060EF7EC1C
:106DD0001FF0010E01D0000E1200FFFFCBD72601DD
:106DE000FFFF04D00101262B000E272326C1F6FF4A
:106DF00027C1F7FF050EF76404D00800FFFFF55028
:106E000005D0F6CFE9FFF7CFEAFFEF50200AD8B45C
:106E1000E9D726C1F6FF27C1F7FF050EF76404D0B6
:106E20000800FFFFF55005D0F6CFE9FFF7CFEAFFE6
:106E3000EF50090A0101D8B4D6D7296B2A6B286B09
:106E400026C1F6FF27C1F7FF050EF76404D008003E
:106E5000FFFFF55005D0F6CFE9FFF7CFEAFFEF507F
:106E60002D0AD8A403D0010E282B15D026C1F6FF79
:106E700027C1F7FF050EF76404D00800FFFFF550A7
:106E800005D0F6CFE9FFF7CFEAFFEF502B0AD8A4E1
:106E900005D0010E01012627000E272326C1F6FF8B
:106EA00027C1F7FF050EF76404D00800FFFFF55077
:106EB00005D0F6CFE9FFF7CFEAFFEF50E7EC1FF080
:106EC000D8A027D00A0E026E036A29C100F02AC199
:106ED00001F04DEC39F026C1F6FF27C1F7FF050E92
:106EE000F76404D00800FFFFF55005D0F6CFE9FFA6
:106EF000F7CFEAFFEF500424006E000E0520016E6C
:106F0000D00E00240101296FFF0E01202A6F010E0F
:106F1000C2D70101285129C100F02AC101F0D8B41B
:106F200005D0001E011E002AD8B4012A1200FFFF5E
:106F300058D77A01FFFF01017E51006E7F51016E2B
:106F40007E07000E7F5B01500010D8B464D07AC178
:106F5000F6FF7BC1F7FF050EF76404D00800FFFFC2
:106F6000F55005D0F6CFE9FFF7CFEAFFEF50000963
:106F7000D8B424D07CC1F6FF7DC1F7FF050EF764BD
:106F800004D00800FFFFF55005D0F6CFE9FFF7CF9A
:106F9000EAFFEF50006E7AC1F6FF7BC1F7FF050EE6
:106FA000F76404D00800FFFFF55005D0F6CFE9FFE5
:106FB000F7CFEAFFEF500018D8B426D07AC1F6FF19
:106FC0007BC1F7FF050EF76404D00800FFFFF55002
:106FD00005D0F6CFE9FFF7CFEAFFEF50006E016A68
:106FE0007CC1F6FF7DC1F7FF050EF76404D00800F1
:106FF000FFFFF55005D0F6CFE9FFF7CFEAFFEF50DE
:10700000005E000E015A09D001017A2B000E7B238D
:107010007C2B7D2390D7006A016A1200FFFF8BD77B
:107020000601FFFF06C1D9FF07C1DAFF01010B51BD
:107030000A11D8B420D00A07D8A00B0708C1F6FF60
:1070400009C1F7FF082B000E0923D9CFE9FFDACFDA
:10705000EAFFD94ADA2A050EF76403D00800F55092
:1070600005D0F6CFE1FFF7CFE2FFE750EF6EEF502C
:10707000D8A4DCD701010A51006E0B51016E0A073A
:10708000000E0B5B01500010D8B408D0D9CFE9FF37
:10709000DACFEAFFD94ADA2AEF6AECD706C100F064
:1070A00007C101F01200FFFFBDD74601FFFF48C135
:1070B000F3FF49C1F4FF46C1D9FF47C1DAFF01011F
:1070C0004A51006E4B51016E4A07000E4B5B015056
:1070D0000010D8B41AD0F3CFF6FFF4CFF7FFF32A9D
:1070E000000EF422D9CFE9FFDACFEAFFD94ADA2A33
:1070F000050EF76403D00800F55005D0F6CFE1FF88
:10710000F7CFE2FFE750EF6EDAD746C100F047C194
:1071100001F01200FFFFCBD7066A046A056A02502D
:10712000031003E1006A016A000C1F0E0612D890DA
:10713000062A02360336FCE3033202320250005CB8
:107140000350015804E3016E0250005ED8800436FB
:107150000536062E06BAF0D706AE05D0041E042A60
:10716000D8B40506051E0450026E0550036E06AC29
:10717000000C001E002AD8B40106011E000C7A0182
:10718000FFFF7AC1F3FF7BC1F4FFF3CFF6FFF4CF2B
:10719000F7FFF32A000EF422050EF76404D008006E
:1071A000FFFFF55005D0F6CFE9FFF7CFEAFFEF502C
:1071B0000009D8A4EAD7F3CF00F0F4CF01F0010121
:1071C0007A51005E7B51015AFF0E0024006EFF0EC3
:1071D0000120016E1200FFFFD4D7FFFF0BD05E0E1F
:1071E000D66EF80ED76E070ED56ED58EF284F28A63
:1071F0001200FFFFF4D7FFFF07D07BC200F07CC274
:1072000001F000D01200FFFFF8D7FFFF11D0F2A469
:1072100001D001D00BD0F80ED76E5E0ED66E0201F3
:10722000010E7B27000E7C238978F2941200FFFF69
:10723000EED7FFFF23D00101026F17D0040E01012A
:10724000016F0CD0500E0101036F03D0010E01013C
:10725000036F01D000D00101032FFCD7010101070A
:107260000129D8A401D001D0EDD7010102070229DC
:10727000D8A401D001D0E2D71200FFFFDCD7EFCFB6
:1072800000F0EE2AEFCF01F0000EEE22EFCF02F079
:10729000EE22EFCF03F0EE22120002500002F3CFF5
:1072A00004F0F4CF05F00102F3500526035000026C
:1072B000F350052612000900F5CFEEFFEA50E26216
:0A72C000FAD7E950E162F7D7120097
:020000040030CA
:04000000FFFAFCFE09
:020000040000FA
:00000001FF
